:100000000C94C60C0C94E50C0C94E50C0C94E50CCB
:100010000C94E50C0C94E50C0C94E50C0C94E50C9C
:100020000C94E50C0C94E50C0C94E50C0C94E50C8C
:100030000C94E50C0C94E50C0C94E50C0C94E50C7C
:100040000C94430F0C94E50C0C94E50C0C94E50C0B
:100050000C94E50C0C94170F0C94E50C0C94E50C27
:100060000C94E50C0C94E50C0C94C40F0C94E50C6A
:100070000C94E50C0C94E50C0C94E50C0C94E50C3C
:100080000C94E50C0C94E50C0C94E50C0C94E50C2C
:100090000C94E50C4C696E65206E756D626572207E
:1000A0006F7574206F662072616E676500000000D6
:1000B00000000000000000000000000053796E7492
:1000C0006178206572726F7200000000000000000D
:1000D0000000000000000000000000000000000020
:1000E00000000000496E76616C696420657870726A
:1000F000657373696F6E000000000000000000006F
:10010000000000000000000000000000556E626169
:100110006C616E63656420706172656E73000000CF
:1001200000000000000000000000000000000000CF
:1001300000000000446174612074797065206D696D
:10014000736D61746368000000000000000000002F
:10015000000000000000000000000000496C6C6519
:1001600067616C206F70657261746F7200000000CF
:10017000000000000000000000000000000000007F
:1001800000000000496C6C6567616C2076617269E3
:1001900061626C65000000000000000000000000CB
:1001A000000000000000000000000000496C6C65C9
:1001B00067616C20746F6B656E2028696E74657260
:1001C0006E616C206572726F722900000000000081
:1001D000000000004F7574206F66206D656D6F72B2
:1001E0007900000000000000000000000000000096
:1001F000000000000000000000000000496E74656F
:10020000676572206F766572666C6F77000000001C
:1002100000000000000000000000000000000000DE
:1002200000000000496E76616C6964206865782082
:1002300064696769740000000000000000000000AD
:100240000000000000000000000000004865782069
:100250006E756D626572206F766572666C6F770081
:10026000000000000000000000000000000000008E
:10027000000000004D697373696E672071756F74BB
:100280006500000000000000000000000000000009
:1002900000000000000000000000000045787065CC
:1002A00063746564206F70656E206F7220636C6F7D
:1002B000736520706172656E000000000000000030
:1002C00000000000274F4E272073796E746178205C
:1002D0006572726F720000000000000000000000F4
:1002E0000000000000000000000000004D69737372
:1002F000696E67205448454E20696E204946207338
:10030000746174656D656E7400000000000000008B
:10031000000000004D697373696E6720544F2069B7
:100320006E20464F522073746174656D656E740063
:100330000000000000000000000000004C696E6535
:10034000206E756D626572206572726F72000000BA
:10035000000000000000000000000000000000009D
:1003600000000000496C6C6567616C206461746119
:10037000207479706500000000000000000000009B
:1003800000000000000000000000000045787072CE
:10039000657373696F6E20746F6F20636F6D706C1F
:1003A0006578000000000000000000000000000070
:1003B000000000004D697373696E6720636F6D6D97
:1003C00061000000000000000000000000000000CC
:1003D0000000000000000000000000004D69737381
:1003E000696E6720636F6D6D61206F722073656D3C
:1003F00069636F6C6F6E0000000000000000000079
:10040000000000004D61746820737461636B206F9D
:10041000766572666C6F77000000000000000000D7
:10042000000000000000000000000000556E64693C
:100430006D656E73696F6E656420617272617900BB
:1004400000000000000000000000000000000000AC
:1004500000000000537562736372697074206F75D9
:1004600074206F662072616E6765000000000000F6
:1004700000000000000000000000000044697669F0
:100480006465206279207A65726F000000000000C8
:10049000000000000000000000000000000000005C
:1004A000000000004C696E65206E6F7420666F75E9
:1004B0006E6400000000000000000000000000006A
:1004C000000000000000000000000000546F6F20DA
:1004D0006D616E79206E657374656420474F535566
:1004E0004273000000000000000000000000000057
:1004F0000000000052455455524E20776974686FD1
:10050000757420474F535542000000000000000062
:10051000000000000000000000000000546F6F2089
:100520006D616E7920616374697665205748494C26
:100530004573000000000000000000000000000003
:1005400000000000454E44574820776974686F7575
:1005500074205748494C450000000000000000008E
:100560000000000000000000000000004F4E20616D
:100570007267756D656E74206D7573742062652089
:100580003E207A65726F000000000000000000004D
:10059000000000004E6F6E73756273637269707451
:1005A000207661726961626C6520696E2044494DF4
:1005B00000000000000000000000000056617269A9
:1005C00061626C6520616C72656164792044494D9B
:1005D000656E73696F6E65640000000000000000C6
:1005E00000000000546F6F206D616E7920616374AC
:1005F00069766520464F522D4E455854206C6F6FDA
:100600007073000000000000000000004E455854C8
:1006100020646F6573206E6F74206D617463682051
:10062000464F5200000000000000000000000000E3
:100630000000000043616E277420434F4E54696EE2
:1006400075650000000000000000000000000000D0
:100650000000000000000000000000004F75742042
:100660006F66206461746120696E205245414420A8
:100670006F7220524553544F524500000000000055
:10068000000000004E6567617469766520737562CD
:10069000736372697074206E6F7420616C6C6F7715
:1006A000656400000000000000000000496C6C65FB
:1006B00067616C20454550282920617267756D651A
:1006C0006E74000000000000000000000000000048
:1006D000000000004F6E6C7920616C6C6F77656470
:1006E00020696E205052494E542073746174656DB8
:1006F000656E740000000000000000004172677524
:100700006D656E74206F7574206F662072616E6700
:100710006520696E20544142000000000000000086
:1007200000000000546F6F206D616E792061726768
:10073000756D656E747320696E2043414C4C0000EA
:10074000000000000000000000000000417275671A
:100750006D656E7420746F2074696D65242829207E
:10076000697320756E6B6E6F776E0000000000007D
:10077000000000002D2D203435202D2D000000001C
:100780000000000000000000000000000000000069
:100790000000000000000000000000002D2D2034AB
:1007A00036202D2D00000000000000000000000099
:1007B0000000000000000000000000000000000039
:1007C000000000002D2D203437202D2D00000000CA
:1007D0000000000000000000000000000000000019
:1007E0000000000000000000000000002D2D20345B
:1007F00038202D2D00000000000000000000000047
:1008000000000000000000000000000000000000E8
:10081000000000002D2D203439202D2D0000000077
:1008200000000000000000000000000000000000C8
:100830000000000000000000000000002D2D203509
:1008400030202D2D000000000000000000000000FE
:100850000000000000000000000000000000000098
:10086000000000002D2D203531202D2D000000002E
:100870000000000000000000000000000000000078
:100880000000000000000000000000002D2D2035B9
:1008900032202D2D000000000000000000000000AC
:1008A0000000000000000000000000000000000048
:1008B000000000002D2D203533202D2D00000000DC
:1008C0000000000000000000000000000000000028
:1008D0000000000000000000000000002D2D203569
:1008E00034202D2D0000000000000000000000005A
:1008F00000000000000000000000000000000000F8
:10090000000000004E6F7420656E6F7567682045AB
:100910004550524F4D20666F72207361766500001E
:10092000000000000000000000000000537461633C
:100930006B20756E646572666C6F77000000000056
:1009400000000000000000000000000000000000A7
:10095000000000005573657220656E7465726564F1
:1009600020425245414B0000000000000000000002
:1009700000000000000000000000000043616E273E
:10098000742075736520414444522077697468204F
:10099000636F6E7374616E740000000000000000ED
:1009A000000000004E6F7420656E6F7567682066EA
:1009B0006C61736820666F72207361766500000059
:1009C0000000000000000000000000002000000007
:1009D0000000000000000000000000000000000017
:1009E0000000000000000000000000000000000007
:1009F00000000000000020000000000000000000D7
:100A0000A939636872240000000000002434737167
:100A100072740000000000008C35616273000000F9
:100A200000000000C733726E640000000000000088
:100A30005D3573676E00000000000000B43974611A
:100A40006200000000000000000020000000000024
:100A5000000000003D357065656B0000000000007F
:100A6000FE34656570000000000000005D396865B7
:100A700078000000000000000000200000000000DE
:100A8000000000009E396865783200000000000018
:100A900083396865783400000000000020357065F7
:100AA000656B31360000000002357065656B3332CE
:100AB000000000005A35616464720000000000000C
:100AC000FA3465657031360000000000F634656563
:100AD0007033320000000000000020000000000021
:100AE000000000005A386C6574000000000000002F
:100AF0005A3800000000000000000000BF3970728A
:100B0000696E740000000000F83D666F720000001E
:100B100000000000BF3B6E6578740000000000001C
:100B20002C3974726F6E000000000000303974724E
:100B30006F666600000000000A37706F6B6500008A
:100B4000000000005A3A64696D00000000000000D7
:100B5000A83672656D000000000000000000200053
:100B60000000000000000000B43664617461000001
:100B700000000000823D726561640000000000001A
:100B8000043B726573746F72650000000000676F4C
:100B900073756200000000000000280000000000E3
:100BA000000000000000290000000000000000001C
:100BB0000138676F746F00000000000009376F6E26
:100BC0000000000000000000F23672657475726E5D
:100BD00000000000953C6966000000000000000075
:100BE000B03D696E7075740000000000DD377374ED
:100BF0006F700000000000007A37656E640000002E
:100C0000000000008D377768696C65000000000007
:100C10000B37656E6477680000000000913C6565E5
:100C200070000000000000008D3C656570313600EA
:100C300000000000893C6565703332000000000050
:100C40000000200000000000000000000000200064
:100C50000000000000000000E931616E6400000047
:100C6000000000000B326F72000000000000000066
:100C70002D32656F72000000000000009F3B696E1E
:100C80006279746500000000000020000000000090
:100C900000000000F63A6F6E74696D650000000098
:100CA000F73A6F6E6972710000000000F83A7265E1
:100CB0007469000000000000F93A6F6E70616363B0
:100CC000000000003339736C65657000000000009F
:100CD00000002000000000000000000000002000D4
:100CE00000000000000000000000200000000000E4
:100CF00000000000000020000000000000000000D4
:100D000000002000000000000000000000002000A3
:100D1000000000000000000029313C00000000003D
:100D200000000000FD303E00000000000000000058
:100D3000D1303C3D0000000000000000A5303E3DE9
:100D4000000000000000000079303D0000000000BD
:100D5000000000004D303C3E00000000000000009C
:100D60000000200000000000000000000000746F80
:100D7000000000000000000000007468656E0000C4
:100D8000000000000000656C7365000000000000BA
:100D90000000737465700000000000000000200077
:100DA0000000000000000000000020000000000023
:100DB0000000000000002000000000000000000013
:100DC00000002000000000000000000000002000E3
:100DD0000000000000000000C7312B0000000000F0
:100DE00000000000A5312D00000000000000000000
:100DF00000002B000000000000000000BF393F0091
:100E00000000000000000000A836270000000000DD
:100E100000000000000020000000000000000000B2
:100E20000000200000000000000000000000200082
:100E30000000000000000000000020000000000092
:100E40000000000000002000000000000000000082
:100E50000000200000000000000000000000200052
:100E60000000000000000000000020000000000062
:100E70000000000000002000000000000000000052
:100E80000000200000000000000000000000200022
:100E9000000000000000000055312A0000000000A2
:100EA0000000000056322F0000000000000000008B
:100EB0007D316D6F64000000000000000000200024
:100EC0000000000000000000000020000000000002
:100ED00000000000000020000000000000000000F2
:100EE00000002000000000000000000000002000C2
:100EF00000000000000000000000200000000000D2
:100F000000000000000020000000000000000000C1
:100F10000000200000000000000000000000200091
:100F200000000000000000000000200000000000A1
:100F30000000000000002000000000000000000091
:100F40000000200000000000000000000000200061
:100F50000000000000000000E22F5E000000000022
:100F60000000000000002000000000000000000061
:100F70000000200000000000000000000000200031
:100F80000000000000000000000020000000000041
:100F90000000000000002000000000000000000031
:100FA0000000200000000000000000000000200001
:100FB0000000000000000000000020000000000011
:100FC0000000000000002000000000000000000001
:100FD00000002000000000000000000000002000D1
:100FE00000000000000000000000200000000000E1
:100FF00000000000000020000000000000000000D1
:1010000000002000000000000000000000002000A0
:101010000000000000000000532F4000000000000E
:1010200000000000A32F6E6F74000000000000009D
:10103000C02F2D0000000000000000000B2F4033E7
:1010400032000000000000007B2F4031360000001D
:101050000000000000002000000000000000000070
:101060000000200000000000000000000000200040
:10107000000000000000000000002300000000004D
:101080000000000000003D00000000000000000023
:1010900001273A00000000000000000000003B00B3
:1010A000000000000000000000002C000000000014
:1010B0000000000000002000000000000000000010
:1010C00000002000000000000000000000002000E0
:1010D000000000000000000074696D6572300000BF
:1010E00000000000000000F0FF0474696D657231BB
:1010F000000000000000000000F1FF0474696D654D
:101100007232000000000000000000F2FF04746969
:101110006D657233000000000000000000F3FF0462
:10112000665F63707500000000000000000000F4BE
:10113000FF04706F72746100000000000000000086
:1011400000220001706F7274620000000000000055
:10115000000000250001706F727463000000000041
:101160000000000000280001706F7274640000002D
:10117000000000000000002B0001646472610000A8
:1011800000000000000000000021000164647262A1
:101190000000000000000000000000240001646462
:1011A0007263000000000000000000000027000142
:1011B0006464726400000000000000000000002A67
:1011C000000170696E610000000000000000000076
:1011D0000020000170696E62000000000000000045
:1011E00000000023000170696E6300000000000031
:1011F000000000000026000170696E64000000001D
:101200000000000000000029000161646373726146
:101210000000000000000000007A000161646D75AC
:1012200078000000000000000000007C0001616404
:10123000636C000000000000000000000078000166
:101240006164636800000000000000000000007995
:101250000001616463000000000000000000000065
:10126000007800027370737200000000000000003C
:101270000000004D00017370647200000000000067
:1012800000000000004E0001737063720000000057
:10129000000000000000004C0001757074696D656D
:1012A000000000000000000000FFFF04706F727477
:1012B00065000000000000000000002E0001706FBB
:1012C00072746600000000000000000000310001A0
:1012D000706F7274670000000000000000000034AE
:1012E000000164647265000000000000000000005E
:1012F000002D000164647266000000000000000020
:10130000000000300001646472670000000000000B
:10131000000000000033000170696E6500000000ED
:10132000000000000000002C000170696E660000E3
:101330000000000000000000002F000170696E67CF
:10134000000000000000000000000032000100006A
:10135000000000000000000000000000000000008D
:10136000000000000000000000000000000000007D
:101370000000000A0D6F72202765652720746F201A
:101380006C6F61642066726F6D20454550524F4D01
:101390002E00556E6B6E6F776E20617267756D658E
:1013A0006E7420746F204C4F41443B207573652050
:1013B00027666C3C6E3E2720746F206C6F61642042
:1013C00066726F6D20464C41534800206461746121
:1013D0002062797465732066726F6D2045455052A6
:1013E0004F4D2E002070726F6772616D20627974AC
:1013F000657320616E6420004C6F61646564200039
:10140000546869732077696C6C206F7665727772A7
:10141000697465207468652063757272656E7420E6
:1014200070726F6772616D20696E2052414D21208C
:101430002041726520796F7520737572653F2000B9
:101440000A0D4E6F2070726F6772616D2073617646
:10145000656420696E20454550524F4D21002E0095
:101460004E6F207375636820666C617368206669CF
:101470006C653B206D757374206265203020746F3D
:1014800020002E00206461746120627974657320ED
:1014900066726F6D20666C6173682066696C65208A
:1014A000002070726F6772616D20627974657320BD
:1014B000616E6420004C6F6164656420005468694B
:1014C000732077696C6C206F7665727772697465CA
:1014D000207468652063757272656E742070726F17
:1014E0006772616D21202041726520796F752073CC
:1014F0007572653F20000A0D4E6F2070726F677223
:10150000616D20736176656420696E20666C61731D
:10151000682066696C6520000A0D6F72202765657A
:101520002720746F207361766520746F20454550C5
:10153000524F4D2E00556E6B6E6F776E2061726745
:10154000756D656E7420746F20534156453B207550
:1015500073652027666C3C6E3E2720746F20736194
:10156000766520746F20464C415348004E6F2070C2
:10157000726F6772616D20696E2052414D3B206E23
:101580006F7468696E672073617665642E002064ED
:1015900061746120627974657320746F20454550D1
:1015A000524F4D2E002070726F6772616D2062790C
:1015B00074657320616E6420005361766564200059
:1015C000546869732077696C6C206572617365205B
:1015D0007468652070726F6772616D206E6F77201E
:1015E000696E20454550524F4D21202041726520A3
:1015F000796F7520737572653F2000206461746196
:1016000020627974657320746F20666C6173682042
:1016100066696C6520002070726F6772616D206270
:101620007974657320616E6420005361766564206F
:101630000021202041726520796F752073757265D5
:101640003F2000546869732077696C6C2065726173
:101650007365207468652070726F6772616D206EAB
:101660006F7720696E20666C6173682066696C65AF
:101670002000206D61726B656420666F7220617559
:10168000746F73746172742E0050726F6772616D43
:1016900020696E20666C6173682066696C65200045
:1016A0000A0D4E6F2070726F6772616D20736176E4
:1016B000656420696E20666C6173682066696C657C
:1016C000200050726F6772616D20696E2045455031
:1016D000524F4D206D61726B656420666F722061A0
:1016E00075746F73746172742E004E6F2070726F18
:1016F0006772616D20736176656420746F20454563
:1017000050524F4D21004175746F73746172742093
:10171000666C61672072656D6F7665642E000A0DD8
:101720004B4C426173696320666F722041746D6532
:101730006C20415652204154393043414E313238A9
:101740002076302E38000A0D436F7265207772695B
:101750007474656E206279204B61726C204C756EDA
:10176000742C206261736564206F6E20476F726411
:101770006F6E20446F7567686D616E2773204241FC
:101780005349433131000A0D4B4C42617369632068
:10179000636F72652076302E39000A0D5245414440
:1017A00059003A20004552524F522023005E5E5E9F
:1017B000003A200020696E206C696E652000455259
:1017C000524F522023000A0D4E6F2070726F6772C5
:1017D000616D20696E206D656D6F72792E000A0D46
:1017E00050726F6772616D206572617365642E005F
:1017F0000A0D546869732077696C6C206572617397
:1018000065207468652063757272656E74207072ED
:101810006F6772616D21202041726520796F75209C
:10182000737572653F20004E6F2070726F67726132
:101830006D206C6F6164656420696E206D656D6FED
:1018400072792E0A0D006461746100270072656D63
:10185000004E6F207375636820666C617368206644
:10186000696C652E00204E6F2070726F6772616D1B
:101870002E003A2000666C00206279746573206641
:101880007265650044796E616D6963206D656D6F89
:10189000727920706F6F6C20286172726179732980
:1018A0003A2000206279746573206672656500567F
:1018B00061726961626C65206D656D6F72793A2045
:1018C0000020627974657320667265650050726FDE
:1018D0006772616D206D656D6F72793A2000556E8B
:1018E0006B6E6F776E204155544F53542061726771
:1018F000756D656E742E20204D75737420626520A1
:101900004F46462C2045452C20464C302C20464C3A
:10191000312C206F7220464C322E00496C6C65676A
:10192000616C206175746F73746172742076616C80
:10193000756520004175746F7374617274206672EE
:101940006F6D20666C61736820004175746F7374ED
:101950006172742066726F6D20454550524F4D2E56
:10196000004175746F7374617274206E6F742065BA
:101970006E61626C65642E000A0D53746F70706541
:1019800064206174206C696E6520000011241FBE04
:10199000CFEFD0E1DEBFCDBF13E0A0E0B1E0E6E3E2
:1019A000FFE700E00BBF02C007900D92A431B10722
:1019B000D9F71FE0A4E1B3E001C01D92AC3FB1072D
:1019C000E1F70E942A180C94993F0C9400002CE730
:1019D0003EE03093C0052093BF0530934F0F209316
:1019E0004E0F83E49FE090934C0C80934B0CF901D5
:1019F00001C0119280914B0C90914C0C8E179F0757
:101A0000C0F786E696E09093570C8093560C90931F
:101A100073058093720581E49CE09093450C80935C
:101A2000440C08959C01220F331FF90143E0EE0F8F
:101A3000FF1F4A95E1F7E20FF31FE951FF4E659151
:101A40007491CB014096049750F4862F8F7090E0EC
:101A5000880F991F880F991F875E9C4F06C08FEFD4
:101A60006F3F780741F485E193E09C01442737FDFF
:101A70004095542F0CC08FEF643F780729F420E085
:101A800030E040E050E003C09B0140E050E0B9018D
:101A9000CA0108959C012458314FC9010895FC01E1
:101AA000DB018CEE9CE09183808380E991E08D9353
:101AB0009C930895FC0110821182128260E070E014
:101AC00080E090E008950895FC0181E0878383839E
:101AD00081E090E091878087148280E790E0968390
:101AE000858360E070E080E090E008950895809143
:101AF000C00085FFFCCF8DE08093C6008091C000C0
:101B000085FFFCCF8AE08093C6000895982F882334
:101B1000C1F180911403882341F19636E1F09736A4
:101B200038F4923681F0953651F09136A9F40DC013
:101B3000923779F0943729F09E3671F408C09BE112
:101B40000BC099E009C098E007C097E005C09AE093
:101B500003C09DE001C09CE0109214038091C0007E
:101B600085FFFCCF9093C60008959C3521F481E059
:101B70008093140308958091C00085FFFCCF90935B
:101B8000C6000895CF93DF93EC0102C00E94860D3A
:101B9000FE01219684918823C9F7DF91CF910895A2
:101BA0008EE197E10E94C20D0895CF93DF93EC017F
:101BB00002C00E94860D89918823D9F7DF91CF91C9
:101BC0000895982F8091C00085FFFCCF9093C600A8
:101BD00008959091490380914A039817D1F3F8949E
:101BE000E0914A03F0E0E75DFC4F808120914A03D9
:101BF00030E02F5F3F4F2F71307020934A0378946D
:101C00000895FF920F931F93CF93DF93EC0110E0A1
:101C100008E060E2F62E0E94E90D982F8D30A9F4BD
:101C200088838091C00085FFFCCF8AE08093C60046
:101C30008091C00085FFFCCF8DE08093C600DF91CE
:101C4000CF911F910F91FF9008958830B9F411231F
:101C500011F38091C00085FFFCCF0093C6008091F6
:101C6000C00085FFFCCFF092C6008091C00085FFC8
:101C7000FCCF0093C60021971150CDCF8A3059F286
:101C80008091C00085FFFCCF9093C60099931F5FA1
:101C9000C2CF1F93142FFC01EE0FFF1F9F0143E0E3
:101CA000220F331F4A95E1F7E20FF31FE751FF4E72
:101CB00044919C01220F331FF901B3E0EE0FFF1F87
:101CC000BA95E1F7E20FF31FE951FF4EA591B491E8
:101CD000413011F41C931CC0423031F4812F952FF8
:101CE00011969C938E9314C0CD014096049780F476
:101CF000F894EA2FF0E0EF70F070EE0FFF1FEE0F98
:101D0000FF1FE75EFC4F10835183628373837894D7
:101D10001F910895FC01EE0FFF1F9F0143E0220F6A
:101D2000331F4A95E1F7E20FF31FE751FF4E44914D
:101D30009C01220F331FF90183E0EE0FFF1F8A95EC
:101D4000E1F7E20FF31FE951FF4EA591B491413045
:101D500021F48C91282F30E005C0423031F48D9170
:101D60009C919C0140E050E030C0CD01409604972A
:101D700078F4EA2FF0E0EF70F070EE0FFF1FEE0F37
:101D8000FF1FE75EFC4F20813181428153811DC0DE
:101D90008FEFAF3FB80749F4209115033091160338
:101DA000409117035091180310C0A45FBF4F29F052
:101DB00020E030E040E050E008C020915F03309127
:101DC00060034091610350916203B901CA01089513
:101DD000833028F020E030E040E050E010C0E82FF1
:101DE000F0E0EE0FFF1FEE0FFF1FEE5FFE4F808152
:101DF0009181A0E0B0E02227382F492F5A2FB90156
:101E0000CA010895CF93DF93EC01A0E0B0E009C0D0
:101E10006BBFFA01879189934F5F5F4F6F4F7F4F81
:101E20001196A217B307A0F3DF91CF9108951F92E7
:101E30000F920FB60F920BB60F9211248F939F93B0
:101E4000EF93FF938091C600833021F481E080936B
:101E5000510C0EC0E0914903F0E0E75DFC4F808338
:101E60008091490390E001968F71907080934903AF
:101E7000FF91EF919F918F910F900BBE0F900FBE2E
:101E80000F901F9018951F920F920FB60F9211246A
:101E90008F939F93AF93BF938091150390911603F7
:101EA000A0911703B09118030196A11DB11D809355
:101EB000150390931603A0931703B0931803809112
:101EC000190390911A03A0911B03B0911C03009772
:101ED000A105B10559F00197A109B1098093190332
:101EE00090931A03A0931B03B0931C0380911D03CE
:101EF00090911E03A0911F03B09120030097A105AC
:101F0000B10559F00197A109B10980931D03909380
:101F10001E03A0931F03B09320038091210390918F
:101F20002203A0912303B09124030097A105B105DA
:101F300059F00197A109B1098093210390932203DD
:101F4000A0932303B093240380912503909126034B
:101F5000A0912703B09128030097A105B10559F07E
:101F60000197A109B1098093250390932603A093BB
:101F70002703B0932803BF91AF919F918F910F904A
:101F80000FBE0F901F9018951F920F920FB60F92D1
:101F900011240F900FBE0F901F9018959B01BC014C
:101FA000660F771FCB01E3E0880F991FEA95E1F7F1
:101FB000680F791F68527F4EC9010E945F3F0895E4
:101FC000CF92DF92EF92FF920F931F93DF93CF9305
:101FD000CDB7DEB72F970FB6F894DEBF0FBECDBFDB
:101FE000FF24A2E1EA2E6E010894C11CD11CFE9CC4
:101FF0008001112408521F4EC8010E94663F892BA0
:1020000059F0C601B8010E945F3FC6010E949C19A9
:10201000892BA1F4F394EBCF20E030E0C9012F9697
:102020000FB6F894DEBF0FBECDBFCF91DF911F91E9
:102030000F91FF90EF90DF90CF900895E091520CB8
:10204000F091530C83E88193F093530CE093520C7E
:102050008F2D90E00E94EE1821E030E0DFCFCF938B
:10206000DF930E94A818E0915B0CF0915C0C8081DA
:1020700090E0C0970A9718F0C0E0D0E036C020E0AA
:1020800030E011C0C90163E0880F991F6A95E1F73C
:10209000220F331F280F391F240F351F3196F0935D
:1020A0005C0CE0935B0CE0915B0CF0915C0C80812C
:1020B000482F50E0405350404A30510518F3E90191
:1020C0000E94A818C330D10584F080E694E10E94F4
:1020D000C20D62E070E080E090E00E94B0218EE5E9
:1020E00094E10E94C20DCFEFDFEFCE01DF91CF91DF
:1020F00008958F929F92AF92BF92CF92DF92EF920C
:10210000FF920F931F93CF93DF934C01FC01EE0FCF
:10211000FF1FEE0FFF1FE050FF4F80819181A0E075
:10212000B0E0EE24F82E092F1A2F7CE0A72EB12C58
:10213000C12CD12CAE0CBF1CC01ED11ECBBEF501D4
:10214000879196918F5F9F4F61F486EF94E10E9493
:10215000C20DB401882777FD8095982F0E94B02189
:1021600021C12091560C3091570C809172059091AD
:1021700073052817390789F08DEB94E10E94C20D91
:102180008BE493E00E94010E80914B0390E00E944B
:102190004F3F8937910509F005C1CBBEF501A791E5
:1021A000B691AA59B94FB093570CA093560C4EE074
:1021B00050E060E070E0E40EF51E061F171F0BBF35
:1021C000F701479156914A0F5B1F50937305409357
:1021D000720562E070E080E090E0E60EF71E081FF6
:1021E000191F0BBFF701879196918458914F9093D7
:1021F000C0058093BF0562E0A62EB12CC12CD12C66
:10220000EA0CFB1C0C1D1D1D0BBFF701279136911D
:10221000820F931F90934F0F80934E0F64E070E0F6
:1022200080E090E0E60EF71E081F191F0BBFF701B4
:10223000879196918451934F9093B8058093B705F9
:102240005A01AA1ABB0AF401EE0FFF1FEE0FFF1F7F
:10225000EE5FFE4F808191817C0100E010E0502F05
:102260004F2D3E2D222760E070E016C04BBFF901D4
:1022700087918C932F5F3F4F4F4F5F4F222349F43D
:102280000894E11CF11C011D111D502F4F2D3E2DF6
:10229000222711966F5F7F4F6A157B0538F30894EC
:1022A000E11CF11C011D111D502F4F2D3E2D222729
:1022B000A091BF05B091C005C0904E0FD0904F0FB8
:1022C000CA1ADB0A60E070E016C04BBFF9018791C3
:1022D0008C932F5F3F4F4F4F5F4F222349F4089459
:1022E000E11CF11C011D111D502F4F2D3E2D2227E9
:1022F00011966F5F7F4F6C157D0538F30894E11CD4
:10230000F11C011D111D502F4F2D3E2D2227C09174
:10231000B705D091B805CC5EDC40ACEEBCE060E027
:1023200070E016C04BBFF90187918C932F5F3F4F30
:102330004F4F5F4F222349F40894E11CF11C011D0B
:10234000111D502F4F2D3E2D222711966F5F7F4F6D
:102350006C177D0738F30E94C02D9093510F809326
:10236000500F85EB94E10E94C20DB50180E090E032
:102370000E94B02181EA94E10E94C20DB60180E082
:1023800090E00E94B02184E894E10E94C20DB40163
:10239000882777FD8095982F0E94B02182E894E1EC
:1023A0000E94C20DDF91CF911F910F91FF90EF908E
:1023B000DF90CF90BF90AF909F908F900895EF9255
:1023C000FF920F931F937C010E94813F182F00E022
:1023D000C70101960E94813F080F111DC8011F917E
:1023E0000F91FF90EF900895AF92BF92CF92DF923E
:1023F000EF92FF920F931F93CF93DF938CE090E0C7
:102400000E94DF118F5F9F4F19F480E494E191C027
:102410002091560C3091570C809172059091730564
:102420002817390789F080E094E10E94C20D8BE4FF
:1024300093E00E94010E80914B0390E00E944F3F79
:102440008937910509F077C08CE090E00E94DF1198
:10245000B6E6CB2EB6E0DB2EC80ED91ED092570CB6
:10246000C092560C8EE090E00E94DF117601E80EDB
:10247000F91EF0927305E092720580E190E00E94EF
:10248000DF118C010458114F1093C0050093BF0554
:1024900082E190E00E94DF11080F191F10934F0F87
:1024A00000934E0F5701AC18BD08C0E0D0E008C043
:1024B000CE014A960E94813FF60181936F012196D9
:1024C000CA15DB05A8F3E090BF05F090C005C090E9
:1024D0004E0FD0904F0FCE18DF088501065E1F4FBC
:1024E000C0E0D0E009C0C8010E94813FF70181939C
:1024F0007F0121960F5F1F4FCC15DD05A0F30E94D1
:10250000C02D9093510F8093500F88EF93E10E945C
:10251000C20DB50180E090E00E94B02184EE93E10D
:102520000E94C20DB60180E090E00E94B0218BECC9
:1025300093E10E94C20DDF91CF911F910F91FF9007
:10254000EF90DF90CF90BF90AF9008950F931F93BF
:10255000CF93DF930E94A81800915B0C10915C0C44
:10256000F80180818D3071F090E00E944F3F8536F8
:10257000910559F4F801818190E00E944F3F853622
:102580009105F1F40E94F41123C086369105C1F43F
:10259000E8012196F801818190E00E944F3F8C363E
:1025A000910571F42196D0935C0CC0935B0C0E9452
:1025B0002F10FFEF8F3F9F0759F00E94791008C03E
:1025C00082E993E10E94C20D83E793E10E94C20D6C
:1025D000DF91CF911F910F91089588E190E00E94C3
:1025E000813F089588E190E00E94813F8A3579F02B
:1025F0008B3518F4853529F407C08B3559F08C35A7
:1026000061F020E030E00FC00E94F4110AC080E0C9
:1026100090E005C081E090E002C082E090E00E947E
:10262000791021E030E0C9010895CF92DF92EF9256
:10263000FF920F931F93DC01CB016C010E94813F3D
:10264000E82EFF2400E010E0102F0F2DFE2CEE24CA
:10265000C60101960E94813FE80EF11C011D111D6B
:10266000B701C8011F910F91FF90EF90DF90CF90BD
:102670000895AF92BF92CF92DF92EF92FF920F93A5
:102680001F937B018C010E9415135B016C01650196
:10269000BB24AA2482E090E0A0E0B0E0E80EF91E9E
:1026A0000A1F1B1FC801B7010E9415139B01AC0133
:1026B0002A0D3B1D4C1D5D1DB901CA011F910F91D3
:1026C000FF90EF90DF90CF90BF90AF900895AF92C2
:1026D000BF92CF92DF92EF92FF920F931F931092CF
:1026E000490310924A031092510C60E070E080E0C0
:1026F00090E00E9439137B018C0160935F0370931B
:102700006003809361039093620364E070E080E073
:1027100090E00E9439135B016C0160936303709336
:102720006403809365039093660368E070E080E043
:1027300090E00E943913AE0CBF1CC01ED11EA6161D
:10274000B706C806D906C1F080E094E2A4EFB0E075
:1027500080935F0390936003A0936103B09362033F
:1027600080E096E9A0E0B0E0809363039093640377
:10277000A0936503B093660382E08093C00088E96C
:102780008093C10086E08093C200E0905F03F090E8
:102790006003009161031091620320916303309103
:1027A0006403409165035091660363E0220F331F79
:1027B000441F551F6A95D1F7C801B7010E94FE3E1C
:1027C00021501092C5002093C4008CE084BDC80144
:1027D000B70120E038EE43E050E00E94FE3E215079
:1027E00027BD80916E00826080936E001092190365
:1027F00010921A0310921B0310921C0310921D03D7
:1028000010921E0310921F031092200310922103B6
:102810001092220310922303109224031092250396
:1028200010922603109227031092280378941F9188
:102830000F91FF90EF90DF90CF90BF90AF900895F1
:10284000DC01CB010E94813F682F70E080E090E0C6
:1028500008951F93CF93DF93EC01162F0E94813FC1
:10286000181721F0CE01612F0E94893FDF91CF918F
:102870001F910895FF920F931F938C01F62E672FDF
:102880000E942914C80101966F2D0E9429141F91DE
:102890000F91FF9008958F929F92AF92BF92CF9227
:1028A000DF92EF92FF920F931F93DF93CF93CDB7F9
:1028B000DEB764970FB6F894DEBF0FBECDBF8CE0D5
:1028C00090E00E94DF118F5F9F4F81F080EC95E1D7
:1028D0000E94C20DCE0101960E94010E898190E0F6
:1028E0000E944F3F8937910509F09CC08091720585
:1028F000909173052091560C3091570C821B930BCD
:1029000020914E0F30914F0F4091BF055091C0055F
:10291000241B350B820F931F4A96875E9F4030F031
:1029200087E38093460C0E942A227CC088E190E0D5
:102930006FEF0E9429148CE090E060E070E00E944C
:102940003A1460917205709173058091560C9091C4
:10295000570C681B790B8EE090E00E943A1480E1DE
:1029600090E060E070E00E943A1460914E0F709128
:102970004F0F8091BF059091C005681B790B82E1D4
:1029800090E00E943A14E090560CF090570C809022
:102990007205909073058E189F0800E010E009C042
:1029A000C8014A96F70161917F010E9429140F5FC7
:1029B0001F4F08151905A0F3C090BF05D090C005A2
:1029C000A0904E0FB0904F0FAC18BD087AE1E72EE3
:1029D000F12CE80CF91C00E010E00BC0C701F60177
:1029E00061916F010E9429140F5F1F4F0894E11C31
:1029F000F11C0A151B0590F389EB95E10E94C20DAD
:102A0000B40180E090E00E94B02185EA95E10E9447
:102A1000C20DB50180E090E00E94B0218EE895E102
:102A20000E94C20D64960FB6F894DEBF0FBECDBFF4
:102A3000CF91DF911F910F91FF90EF90DF90CF909A
:102A4000BF90AF909F908F900895CF92DF92EF92BA
:102A5000FF920F931F93CF93DF932091560C3091E9
:102A6000570C80917205909173052817390719F456
:102A70008CE695E1C7C10E94A81800915B0C1091EB
:102A80005C0CD8018C918D3079F090E00E944F3F22
:102A90008536910561F4F801818190E00E944F3FF5
:102AA0008536910509F0A8C10E944B14ADC1863648
:102AB000910509F0A1C1E8012196D80111968C91E8
:102AC00090E00E944F3F8C36910509F095C1219608
:102AD000D0935C0CC0935B0C0E942F106C01BFEF75
:102AE0008F3F9B0709F490C1FC01EE0FFF1FEE0F13
:102AF000FF1FE050FF4F80819181A0E0B0E0EE2405
:102B0000F82E092F1A2F2CE030E040E050E0E20EC2
:102B1000F31E041F151F0BBFF7018791969124EF39
:102B20003FEF4FEF5FEFE20EF31E041F151F8F5FA5
:102B30009F4FE1F083E496E10E94C20DB601882721
:102B400077FD8095982F0E94B02181E396E10E9445
:102B5000C20D8BE493E00E94010E80914B0390E044
:102B60000E944F3F8937910509F04EC120917205AF
:102B7000309173056091560C7091570C922F961BF3
:102B800040914E0F50914F0FE091BF05F091C0055D
:102B9000A42FAE1B892F8A0F865E80935F0C8FEF68
:102BA00080937F03109273031092740390937503C4
:102BB000261B370B3093760310927703109278031D
:102BC000A09379034E1B5F0B50937A0310927B0303
:102BD00010927C038091B7059091B8052CEE3CE0F3
:102BE000482F421B40937D038C5E9C40892F990F98
:102BF000990B80937E03C801B70147E653E00E941A
:102C000000FEF601EE0FFF1FEE0FFF1FEE5FFE4FFF
:102C1000808191817C0100E010E0C0E0D0E040E0E4
:102C200050E01EC0FA01E959FC4FDE01AA59B94F24
:102C30008C9180834F5F5F4F81E04030580779F47B
:102C4000902F8F2D7E2D662747E653E00E9400FED1
:102C50000894E11CF11C011D111D40E050E021967B
:102C600080917205909173052091560C3091570C0C
:102C7000821B930BC817D907A8F2452B41F0902F60
:102C80008F2D7E2D662747E653E00E9400FE0894B4
:102C9000E11CF11C011D111DC0E0D0E040E050E03E
:102CA0001EC0FA01E959FC4FDE01A458B14F8C91C6
:102CB00080834F5F5F4F91E04030590779F4902F48
:102CC0008F2D7E2D662747E653E00E9400FE089474
:102CD000E11CF11C011D111D40E050E02196809186
:102CE0004E0F90914F0F2091BF053091C005821B70
:102CF000930BC817D907A8F2452B41F0902F8F2DC1
:102D00007E2D662747E653E00E9400FE0894E11CF2
:102D1000F11C011D111DC0E0D0E020E030E01EC01C
:102D2000F901E959FC4FDE01A451B34F8C91808326
:102D30002F5F3F4FA1E020303A0779F4902F8F2D7D
:102D40007E2D662747E653E00E9400FE0894E11CB2
:102D5000F11C011D111D20E030E021968091B70586
:102D60009091B8058C5E9C40C817D907C8F2232BF8
:102D700041F0902F8F2D7E2D662747E653E00E946D
:102D800000FE8AE296E10E94C20D60917205709188
:102D900073052091560C3091570C621B730B8827DA
:102DA00077FD8095982F0E94B02186E196E10E94E0
:102DB000C20D60914E0F70914F0F2091BF05309161
:102DC000C005621B730B882777FD8095982F0E94A2
:102DD000B0218BEF95E10E94C20DB601882777FDE7
:102DE0008095982F0E94B0218091C00085FFFCCF74
:102DF0008EE28093C60008C085E395E10E94C20D73
:102E000088E195E10E94C20DDF91CF911F910F9152
:102E1000FF90EF90DF90CF900895EF92FF920F9385
:102E20001F939C018F3F910541F488E190E06FEF83
:102E30000E94291486E097E15AC08535910591F4E6
:102E40008CE090E00E94DF118F5F9F4F19F48AEEB3
:102E500096E14DC088E190E065E50E94291482EC7E
:102E600096E145C08A35910511F460E00AC08B35C2
:102E7000910511F461E005C08C35910509F039C068
:102E800062E0E62FF0E0EE0FFF1FEE0FFF1FE050B5
:102E9000FF4F80819181A0E0B0E0BA2FA92F982F39
:102EA00088270C96A11DB11DABBFFC01879196919F
:102EB000E62EFF2400E010E08F5F9F4F49F480EA88
:102EC00096E10E94C20DC801B7010E94B02111C055
:102ED00088E190E0622F0E94291489E896E10E941F
:102EE000C20DC801B7010E94B02182E796E10E949D
:102EF000C20D1F910F91FF90EF900895DF92EF9216
:102F0000FF920F931F937B018C01D42ECB01652F71
:102F10000E94893F0894E11CF11CC7016D2D0E949D
:102F2000893F1F910F91FF90EF90DF900895AF922E
:102F3000BF92CF92DF92EF92FF920F931F937B018C
:102F40008C0159016A019A0144275527A9010E9461
:102F50007E1782E090E0A0E0B0E0E80EF91E0A1FC4
:102F60001B1FC801B701A5010E947E171F910F9179
:102F7000FF90EF90DF90CF90BF90AF900895DC016D
:102F8000CB01642F0E94893F08956F927F928F92A8
:102F90009F92BF92CF92DF92EF92FF920F931F9377
:102FA000DF93CF93CDB7DEB72F970FB6F894DEBF80
:102FB0000FBECDBF4C01BB2413E1612E712C6E01FD
:102FC0000894C11CD11C8B2D90E0869D7001879DBB
:102FD000F00C969DF00C11248701005A1C4EC8017C
:102FE0000E94663F892BF9F0C601B8010E945F3F3D
:102FF000C6010E949C19892BA1F0F701E159FC4EF2
:1030000085919591A591B491F40180839183A283D8
:10301000B383F60101900020E9F73197EC19FD091F
:1030200004C0B394D0CFE0E0F0E0CF012F960FB60C
:10303000F894DEBF0FBECDBFCF91DF911F910F91EE
:10304000FF90EF90DF90CF90BF909F908F907F90F8
:103050006F9008950E941D1B81E090E00895FC018F
:1030600011824083738362830895FC01118240833F
:10307000738362830895FC018181882331F4609316
:10308000460C0E942A2280E00895815081830280AC
:10309000F381E02DE80FF11D80810895DC01119688
:1030A0009C9111978C91981729F44093460C0E949B
:1030B0002A2208951296ED91FC911397E90FF11DC4
:1030C000608311968C9111978F5F11968C93089560
:1030D000FC018181882349F46093460C0E942A22D6
:1030E00020E030E040E050E010C08150818390E06B
:1030F000880F991F880F991F0280F381E02DE80F38
:10310000F91F2081318142815381B901CA0108959B
:10311000DC0111963C9111978C91381729F420937A
:10312000460C0E942A220895832F90E0880F991F51
:10313000880F991F1296ED91FC911397E80FF91FD4
:1031400040835183628373833F5F11963C9308955C
:1031500005C03196F0935C0CE0935B0CE0915B0C46
:10316000F0915C0C80818032A1F30895E0915B0CBA
:10317000F0915C0C808190E0C0970A97E8F019C04C
:10318000CA01B3E0880F991FBA95E1F7440F551FA4
:10319000480F591F460F571F3196F0935C0CE09370
:1031A0005B0C4217530710F09A010AC081E080932C
:1031B000460C40E050E010C040E050E020E030E03D
:1031C000E0915B0CF0915C0C8081682F70E06053A3
:1031D00070406A307105A0F2CA010895E091520C66
:1031E000F091530C81939193F093530CE093520C14
:1031F0000895E091520CF091530C918380831282D8
:103200003396F093530CE093520C089590E006C06F
:103210003196F0935C0CE0935B0C9F5FE0915B0C4C
:10322000F0915C0C8081803299F39923C1F0A091D8
:10323000520CB091530C923058F0FD018FE78193FE
:1032400011969C933196F093530CE093520C089591
:10325000FD018EE78193F093530CE093520C089597
:10326000E0915B0CF0915C0C8081089580915B0C87
:1032700090915C0C019690935C0C80935B0C08958C
:10328000E091520CF091530C61937193819391935F
:10329000F093530CE093520C0895282FE091520CB8
:1032A000F091530C809154069091550680589F4F91
:1032B000E817F90721F484E18093460C08952083F0
:1032C0008091520C9091530C01969093530C8093E3
:1032D000520C0895AF92BF92CF92DF92FF920F935C
:1032E0001F93CF93DF935C016B01C0E0D0E013C06C
:1032F000F501EC0FFD1F808190E00E94573F8C018B
:103300008F2D90E00E94573F0817190719F0C0E071
:10331000D0E007C02196F601EC0FFD1FF080FF20E2
:1033200039F7CE01DF91CF911F910F91FF90DF9080
:10333000CF90BF90AF9008950F931F93182F092F30
:1033400080915B0C90915C0C612F702F0E946A1928
:10335000892B19F4A0E0B0E013C0E12FF02FDF01BA
:103360000D900020E9F71197AE1BBF0B80915B0C0D
:1033700090915C0C8A0F9B1F90935C0C80935B0C6C
:10338000CD011F910F91089515C11092B9050E94AA
:1033900006198CE091E00E949C19892B19F00E947B
:1033A000571CF2C081E191E00E949C19892B19F011
:1033B0000E944A1EE9C085E191E00E949C19892B78
:1033C00019F00E943923E0C08AE191E00E949C1923
:1033D000892B19F00E948F21D7C082E291E00E94D0
:1033E0009C19892B19F00E94771ECEC088E291E0CB
:1033F0000E949C19892B19F00E94731EC5C08DE292
:1034000091E00E949C19892B19F00E949A24BCC05B
:1034100080E391E00E949C19892B19F00E94EF1B18
:10342000B3C087E391E00E949C19892B19F00E9498
:103430000424AAC08AE391E00E949C19892B19F008
:103440000E945A23A1C080E491E00E949C19892B1C
:1034500019F00E94EC2298C086E491E00E949C1929
:10346000892B19F00E9494238FC08AE491E00E9476
:103470009C19892B19F00E94462386C08FE491E0A5
:103480000E949C19892B19F00E94FA1B7DC084E5CB
:1034900091E00E949C19892B19F00E949A2174C016
:1034A0008AE591E00E949C19892B19F00E94051C65
:1034B0006BC08EE591E00E949C19892B19F00E9447
:1034C0005F1C62C082E691E00E949C19892B19F072
:1034D0000E94272359C086E691E00E949C19892BFF
:1034E00019F00E94101C50C08BE691E00E949C19BC
:1034F000892B19F00E941B1C47C081E791E00E94B4
:103500009C19892B19F00E9488223EC087E791E020
:103510000E949C19892B19F00E94092635C08DE75D
:1035200091E00E949C19892B19F00E9405262CC05D
:1035300083E891E00E949C19892B19F00E940D26C6
:1035400023C087E891E00E949C19892B19F00E9402
:10355000F0221AC08EE891E00E949C19892B19F084
:103560000E94E82211C080E991E00E949C19892BF9
:1035700019F00E945B1C08C082E991E00E949C192E
:10358000892B91F50E94461E8091460C882361F597
:103590000E940619E0915B0CF0915C0CE081EA332B
:1035A00019F40E94DB1B06C0ED3021F082E080930D
:1035B000460C0895E0915B0CF0915C0C80818D309D
:1035C00009F0E3CEE091520CF091530C8DE780832B
:1035D0008091BE05882341F42091520C88E59FE03C
:1035E000281B2F5F20935A0F08951F93182F90E0E8
:1035F0000E943D3F892B39F420E030E0812F90E09C
:10360000C0970A9710F421E030E0C9011F91089596
:103610000F931F9300E61CE0C8010E94010EF80101
:1036200001900020E9F731978DE0808310935C0CC6
:1036300000935B0C1F910F910895DF92EF92FF9220
:103640000F931F93DF93CF9300D0CDB7DEB70E94C7
:1036500067130E94942D0E947F2D87EB95E0BE0199
:103660006F5F7F4F0E944F0D8091B7059091B80515
:1036700029813A81820F931F90934B0F80934A0FB9
:103680000E94F212892B11F00E945D290E94770D91
:103690000E94770D0E94D00D86E897E10E94C20D2E
:1036A00086E497E10E94C20D81E08093BE0518E593
:1036B000E12E1FE0F12EDD24D3948091BE058823F6
:1036C00021F08AE997E10E94C20D1092BE05109286
:1036D000460C10924E060E94770D8EE30E94E10D7B
:1036E0000E94081B05C03196F0935C0CE0935B0CC4
:1036F000E0915B0CF0915C0C80818032A1F380EE54
:103700009CE069E975E04EE10E94351884EE9CE08A
:103710006BE774E04CE30E942F180E94612C892B08
:1037200061F600914E0F10914F0FF092530CE09202
:10373000520C109298050E94B6189C010097D1F087
:10374000E0915B0CF0915C0C80818D3021F4C9011B
:103750000E94DB2D24C01092BE05E091520CF09126
:10376000530C3183208312823396F093530CE093F1
:10377000520C02C0D092BE058091460C882379F489
:103780000E94C4198091460C882349F48091BE059B
:10379000882319F00E94182702C00E94BF2E809132
:1037A000460C882309F489CF0E942A2210934F0FD8
:1037B00000934E0F82CFE091520CF091530C8AE7A8
:1037C0008193F093530CE093520C80915B0C909199
:1037D0005C0C019690935C0C80935B0C0895E091D7
:1037E000520CF091530C84E18193F093530CE093CD
:1037F000520C0895E091520CF091530C87E18193A3
:10380000F093530CE093520C0895E091520CF09118
:10381000530C88E18193F093530CE093520C08957C
:10382000E091520CF091530C86E08193F093530C8D
:10383000E093520C0895E091520CF091530C87E004
:103840008193F093530CE093520C0895A091520C85
:10385000B091530CFD01819311961C9211973196F2
:10386000F093530CE093520C22E0E0915B0CF0914A
:103870005C0C8191F0935C0CE0935B0CE091520C3A
:10388000F091530C8193F093530CE093520C8D30D4
:1038900011F02F5FEACF80915B0C90915C0C019747
:1038A00090935C0C80935B0C11962C9308958CE0A4
:1038B0000E94261C089584E40E94261C08958AE034
:1038C0000E94261C089587E991E00E949C19892B8B
:1038D00011F082E308958AE991E00E949C19892BF6
:1038E00011F083E308958DE991E00E949C19892BE2
:1038F00011F085E3089580EA91E00E949C19892BDC
:1039000011F080E3089582EA91E00E949C19892BCE
:1039100011F081E3089584EA91E00E949C19892BBB
:1039200011F480E0089584E3089586EA91E00E940E
:103930009C19892B11F080E208958AEA91E00E9497
:103940009C19892B11F081E208958DEA91E00E9483
:103950009C19892B11F480E0089582E2089581EB8F
:1039600091E00E949C19892B11F080E4089583EB6B
:1039700091E00E949C19892B11F081E4089585EB58
:1039800091E00E949C19892B11F080E5089587EB46
:1039900091E00E949C19892B11F081E5089589EB33
:1039A00091E00E949C19892B11F082E508958DEB1E
:1039B00091E00E949C19892B11F480E0089580E623
:1039C00008959F92AF92BF92CF92DF92EF92FF92B3
:1039D0000F931F93182F00E061E7962E50E7B52E46
:1039E00043E7A42E34E7D32E22E7C22E90E1E92E3E
:1039F00081E1F82E0E94061983EB91E00E949C1948
:103A0000892B31F0E091520CF091530CC1922FC0F0
:103A10008FEB91E00E949C19892B31F0E091520CC0
:103A2000F091530CD19223C083EC91E00E949C1939
:103A3000892B31F0E091520CF091530CA19217C0F8
:103A400087EC91E00E949C19892B31F0E091520C97
:103A5000F091530CB1920BC089EC91E00E949C193B
:103A6000892B49F0E091520CF091530C9192F09314
:103A7000530CE093520C0E940619E0915B0CF091FC
:103A80005C0C80818832B9F5E091520CF091530CB6
:103A9000E192F093530CE093520C80915B0C909167
:103AA0005C0C019690935C0C80935B0C812F0E94C0
:103AB000E11C8091460C882309F077C0E0915B0CF3
:103AC000F0915C0C8081893211F084E060C0E0915B
:103AD000520CF091530CF192F093530CE093520C72
:103AE00080915B0C90915C0C019690935C0C8093A0
:103AF0005B0C11E01EC00E94E71F982F882369F419
:103B00000E941126982F882341F40E94E00F982FDD
:103B1000882319F40E94C520982F8091460C882391
:103B200009F043C0112321F0911711F085E02FC057
:103B3000192F0E940619E0915B0CF0915C0CE0815A
:103B4000ED3099F1EA3389F1EC3279F1EB3369F137
:103B5000E93259F11130C1F40E94AF1C8823D9F425
:103B60000E94951C8823B9F48091B905882339F007
:103B70000023D9F40E94631C882361F407C080915C
:103B8000F90F882319F011C083E101C086E080930A
:103B9000460C0BC001E0E091520CF091530C819364
:103BA000F093530CE093520C25CF1F910F91FF908F
:103BB000EF90DF90CF90BF90AF909F9008951F93AC
:103BC0000E94E00F182F882329F40E94C520182F87
:103BD000882311F18091460C8823F1F40E94061984
:103BE000E0915B0CF0915C0C8191F0935C0CE093A4
:103BF0005B0C8D3321F083E08093460C0DC0E09187
:103C0000520CF091530C89E78193F093530CE0939D
:103C1000520C812F0E94E11C1F910895E091520CDB
:103C2000F091530C8193F093530CE093520C0E944B
:103C3000061983EC91E00E949C19892B31F0E091E8
:103C4000520CF091530C83E717C08FEB91E00E9468
:103C50009C19892B31F0E091520CF091530C84E7C0
:103C60000BC087EC91E00E949C19892B51F0E091E8
:103C7000520CF091530C80E78193F093530CE09336
:103C8000520C0E9406190E94DF1D089582E00E94D6
:103C90000E1E089581E00E940E1E0895E091520CC0
:103CA000F091530C8193F093530CE093520C0E94CB
:103CB0000619E091520CF091530C88EA8193F0932D
:103CC000530CE093520C0E94B6189C01009719F413
:103CD00082E18093460C8091460C882319F4C90137
:103CE0000E94EE18089582E10E944E1E08958FE012
:103CF0000E944E1E0895E0915B0CF0915C0C808157
:103D0000883219F424E930E002C020E030E0C90133
:103D10000895282FDB0140914E0F50914F0FFA016B
:103D20008193F0934F0FE0934E0F90E08C91E091D0
:103D30004E0FF0914F0F8193F0934F0FE0934E0F82
:103D40008C91811111969F5F9E3081F7243851F03C
:103D5000243941F0223811F494E005C0213811F0E3
:103D600088E01BC095E081E020914E0F30914F0F0D
:103D7000F9011192F0934F0FE0934E0F8F5F981758
:103D800098F730934F0F20934E0F80914B0C9091EA
:103D90004C0C8217930730F489E08093460CEFEFC8
:103DA000FFEF07C08091BF059091C005FA01E81BA5
:103DB000F90BCF0108950F931F93CF93DF93E091F9
:103DC0005B0CF0915C0C808190E0C0970A9728F41E
:103DD00020E030E040E050E025C082E016C0CA019B
:103DE000B9012AE030E040E050E00E94BF3E9B0174
:103DF000AC01CE01AA2797FDA095BA2F280F391F35
:103E00004A1F5B1F57FF08C08AE08093460C20E0E2
:103E100030E040E050E012C00F5F1F4F10935C0C89
:103E200000935B0C00915B0C10915C0CF80180819D
:103E3000C82FD0E0E097CA30D10588F2B901CA0195
:103E4000DF91CF911F910F910895CF93DF93C09190
:103E5000520CD091530CDE0182EA8D93CD01019674
:103E60009093530C8093520CE0915B0CF0915C0C9E
:103E7000219111962C9301969093530C8093520CA0
:103E8000F0935C0CE0935B0C22E018C08D3019F4C9
:103E90008093460C2DC0E091520CF091530C81930D
:103EA000F093530CE093520C80915B0C90915C0C5E
:103EB000019690935C0C80935B0C2F5FE0915B0C00
:103EC000F0915C0C8081823209F7E091520CF09104
:103ED000530C8193F093530CE093520C80915B0C44
:103EE00090915C0C019690935C0C80935B0C298301
:103EF000DF91CF91089590E00E94443F0895BF92D2
:103F0000CF92DF92EF92FF920F931F93CF93DF93A5
:103F1000E0915B0CF0915C0C808190E00E94443F4A
:103F2000892B29F0EE24FF248701BB2433C08BE0CA
:103F300023C09E0120533040D801C70144E0880FC0
:103F4000991FAA1FBB1F4A95D1F72A30310530F4BB
:103F500079010027F7FC0095102F06C0E7977E0136
:103F60000027F7FC0095102FE80EF91E0A1F1B1FF3
:103F700089E0B81639F48CE08093460CEE24FF24D7
:103F8000870119C0B3940894C11CD11CD0925C0C59
:103F9000C0925B0CC0905B0CD0905C0CF6018081F1
:103FA00090E00E94573FC82FD0E0CE010E94443FCE
:103FB000892B09F0BECFB701C801DF91CF911F91C6
:103FC0000F91FF90EF90DF90CF90BF9008950F93E7
:103FD0001F93DF93CF9300D000D0CDB7DEB7009111
:103FE0005B0C10915C0CF8018081823229F40E94F4
:103FF000251F22E030E04FC0843259F40F5F1F4F7D
:1040000010935C0C00935B0C015010400E947F1FCA
:104010000EC090E00E943D3F892B39F0CE01019601
:104020000E94C517882339F434C00E94DB1E6983BF
:104030007A838B839C838091460C882351F5E09191
:10404000520CF091530C84EA8193F093530CE0935B
:10405000520C69817A818B819C810E9440198091E8
:104060005B0C801B03C0F80181918F01E091520C21
:10407000F091530C8193F093530CE093520C809188
:104080005B0C90915C0C0817190768F321E030E095
:1040900002C020E030E0C9010F900F900F900F9008
:1040A000CF91DF911F910F910895CF93DF93EC0192
:1040B000E881F9818081843981F47396F983E883FA
:1040C000739787859089009701F1DC012D913D91CF
:1040D000220F331F220F331F10C0843841F4DF0139
:1040E0001F967396F983E88324E030E006C088E0E9
:1040F0008093460C0E942A2208C080E090E002C013
:104100001D92019682179307D8F3DF91CF910895FE
:10411000EF92FF920F931F93CF93DF93E82E8B01C3
:10412000FB0101900020E9F73197FE2EF61AC091AD
:10413000BF05D091C0051CC08E1581F4BE016F5F14
:104140007F4FC8010E946A19F81641F48091BF059B
:104150009091C005BE01681B790B0FC0888184381F
:1041600031F0843921F088E08093460C04C06396D6
:104170008881882309F76FEF7FEFCB01DF91CF9123
:104180001F910F91FF90EF9008951F93CF93DF93AE
:10419000E7E6F4E0119284E0E637F807D9F7C0913A
:1041A0005B0CD0915C0C1881812F90E00E943D3F08
:1041B000892B41F0109367042196D0935C0CC09337
:1041C0005B0C03C087E08093460CC8E6D4E0E09126
:1041D0005B0CF0915C0C80810E94F51A892B71F0C8
:1041E000E0915B0CF0915C0C81918993F0935C0CF5
:1041F000E0935B0C84E0C537D80749F7E0915B0C8E
:10420000F0915C0C8081883219F484E990E002C05E
:1042100080E090E080937604882321F484E8809302
:10422000760405C03196F0935C0CE0935B0C8091B2
:10423000460C882309F051C08091760467E674E04B
:104240000E9488209C018091460C882309F045C07B
:104250008FEF2F3F3807C1F490917604943931F4F1
:1042600080919805882311F488E135C0892F67E68D
:1042700074E00E94891E9C018FEF2F3F380769F17F
:104280008091460C882349F580917604E091520C88
:10429000F091530C8193F093530CE093520CC901AD
:1042A0000E94EE1880917604843949F5E091520C11
:1042B000F091530C80E18193F093530CE093520CF6
:1042C00081E00E94E11CE0915B0CF0915C0C80812C
:1042D000893231F08EE08093460C20E030E01AC045
:1042E0003196F0935C0CE0935B0CE091520CF091F2
:1042F000530C81E18193F093530CE093520C809125
:104300007604843829F0843919F022E030E002C0C4
:1043100021E030E0C901DF91CF911F910895E09134
:10432000520CF091530C8EE08193F093530CE09378
:10433000520C0895E091520CF091530C8AE1819354
:10434000F093530CE093520C0895E091520CF091CD
:10435000530C8CE08193F093530CE093520C08952E
:104360008F929F92AF92BF92CF92DF92EF92FF9285
:104370000F931F93DF93CF93CDB7DEB764970FB63C
:10438000F894DEBF0FBECDBF7B018C011C8A97FF66
:1043900011C08DE20E94E10DAA24BB246501AE1874
:1043A000BF08C00AD10A82E1F82E4E010894811C90
:1043B000911C26C0611571058105910519F05B01FD
:1043C0006C01F1CF80E30E94E10D28C0080D191D9A
:1043D000C601B5012AE030E040E050E00E94FE3E18
:1043E000605DF8016083FA94C601B5012AE030E00F
:1043F00040E050E00E94FE3EC901DA015C016D011F
:104400000F2D10E0A114B104C104D104F9F60F5F1F
:104410001F4FC401800F911F0E94D50D64960FB6E7
:10442000F894DEBF0FBECDBFCF91DF911F910F91EA
:10443000FF90EF90DF90CF90BF90AF909F908F90C4
:10444000089598E2899FC001112484599F4F0E94CA
:10445000C20D0895CF93DF9380914E068823D1F04B
:104460008EEB97E10E94C20D6091460C70E080E0F7
:1044700090E00E94B02184EB97E10E94C20D609110
:104480005D0C70915E0C80E090E00E94B02181EBA9
:1044900097E132C00E94770D0E94770DC0E6DCE004
:1044A00002C00E94E10D89918D30D9F70E94770DED
:1044B00020E63CE004C08AE20E94E10D9E01E90191
:1044C000219680915B0C90915C0C0297281739071C
:1044D00090F38DEA97E10E94C20D0E94770D85EA64
:1044E00097E10E94C20D6091460C70E080E090E080
:1044F0000E94B02182EA97E10E94C20D8091460C91
:104500000E94212281E08093430CDF91CF91089596
:104510008091B9058F5F8093B905E091520CF091BD
:10452000530C89E18193F093530CE093520C80E09B
:104530000E94E11C08950F931F93E091520CF0919B
:10454000530C8193F093530CE093520C0E94061984
:104550000BE71CE731C080E00E94E11C8091460C13
:10456000882399F50E940619E0915B0CF0915C0C90
:10457000E081EC3231F4E091520CF091530C108355
:1045800007C0EB3311F5E091520CF091530C00830E
:1045900080915B0C90915C0C019690935C0C8093E5
:1045A0005B0C8091520C9091530C01969093530C9C
:1045B0008093520C0E940619E0915B0CF0915C0C08
:1045C000E081ED3011F0EA3331F61F910F9108953B
:1045D00083E40E949B22089583E00E949B22089519
:1045E000E091520CF091530C83E28193F093530CC1
:1045F000E093520C0E9406190E94C52008951F9353
:104600001CE70E9406190E94C5208091460C882351
:10461000E1F40E940619E0915B0CF0915C0C808142
:104620008C3299F4E091520CF091530C1193F09369
:10463000530CE093520C80915B0C90915C0C0196B2
:1046400090935C0C80935B0CDCCF1F91089581E00C
:1046500080939805E091520CF091530C89E081937E
:10466000F093530CE093520C0E94FF221092980595
:104670000895E091520CF091530C8DE08193F093EA
:10468000530CE093520C0E94FF220895E091520CCB
:10469000F091530C85E08193F093530CE093520C0E
:1046A0000E9406190E94C520019719F082E08093AC
:1046B000460C0895E091520CF091530C86E18193E1
:1046C000F093530CE093520C0E940619E0915B0C9E
:1046D000F0915C0C8081823221F50E94251F80912F
:1046E000460C882301F5E0915B0CF0915C0C808115
:1046F0008C3221F082E08093460C0895E091520CB8
:10470000F091530C8CE78193F093530CE093520C8F
:1047100080915B0C90915C0C019690935C0C809363
:104720005B0C0E94FF2208951F9381E08093F90F94
:10473000E091520CF091530C84E08193F093530C70
:10474000E093520C0E9406190E94C520182F0E9467
:104750000619113059F4E0915B0CF0915C0C8191D9
:10476000F0935C0CE0935B0C8D3311F083E02EC072
:10477000E091520CF091530C89E78193F093530C24
:10478000E093520C81E00E94E11C8091460C88234A
:10479000C9F50E9406198DEC91E00E949C19892BA5
:1047A000A1F0E091520CF091530C87E38193F093C8
:1047B000530CE093520C0E94061981E00E94E11C08
:1047C0008091460C8823F1F404C081E18093460C6B
:1047D00019C00E94061980ED91E00E949C19892B56
:1047E00079F0E091520CF091530C8AE38193F093AD
:1047F000530CE093520C0E94061981E00E94E11CC8
:104800001092F90F1F910895E091520CF091530C02
:1048100085E18193F093530CE093520C0E940619AA
:104820008091B9058F5F8093B90581E00E94E11CFA
:104830008091460C882309F07CC00E94061985ED02
:1048400091E00E949C19892BB9F1E091520CF091F2
:10485000530C88E38193F093530CE093520C0E9425
:104860000619E0915B0CF0915C0C808190E0C097A0
:104870000A97D8F4E091520CF091530C88EA819396
:10488000F093530CE093520C0E94B6189C010097D1
:1048900019F482E18093460C8091460C882309F03C
:1048A00048C0C9010E94EE180BC00E94C419809133
:1048B000460C882329F0089580E18093460C0895E2
:1048C0000E9406198AED91E00E949C19892B89F1BA
:1048D000E091520CF091530C89E38193F093530CC7
:1048E000E093520C0E940619E0915B0CF0915C0C75
:1048F000808190E0C0970A97D0F4E091520CF0913B
:10490000530C88EA8193F093530CE093520C0E946D
:10491000B6189C01009719F482E18093460C8091AF
:10492000460C882331F4C9010E94EE1808950E94B4
:10493000C4190895FF920F931F93E091520CF091C8
:10494000530C83E18193F093530CE093520C0E943B
:10495000061981E00E94E11C8091460C882309F031
:1049600056C00E9406198FED91E00E949C19892B78
:1049700019F00E94731E0CC084EE91E00E949C19F5
:10498000892B19F00E94771E03C08FE08093460C9C
:104990008091460C8823D9F50E9406199CE7F92ED0
:1049A00008EA12E12DC0E091520CF091530CF19203
:1049B000F093530CE093520C80915B0C90915C0C43
:1049C000019690935C0C80935B0C0E940619E09119
:1049D000520CF091530C0193F093530CE093520C52
:1049E0000E94B6189C01009711F41093460C809118
:1049F000460C882361F4C9010E94F9180E94061927
:104A0000E0915B0CF0915C0C80818C3261F21F9123
:104A10000F91FF900895DF92EF92FF920F931F93F3
:104A2000CF93DF938B017A01C091520CD091530C3C
:104A3000DE018D93B093530CA093520CE0915B0C6C
:104A4000F0915C0C8081883239F580E18983119680
:104A5000B093530CA093520C80915B0C90915C0C22
:104A6000019690935C0C80935B0C8CE7D82EF70139
:104A700081917F010E94E11C8091460C8823D9F529
:104A800001501040E0915B0CF0915C0C0115110598
:104A9000C1F080818C3211F082E017C0E091520C9D
:104AA000F091530CD192F093530CE093520C8091FF
:104AB0005B0C90915C0C019690935C0C80935B0C6A
:104AC000D6CF8081893221F08EE08093460C13C0CE
:104AD000E091520CF091530C81E18193F093530CCF
:104AE000E093520C80915B0C90915C0C019690933A
:104AF0005C0C80935B0CDF91CF911F910F91FF9025
:104B0000EF90DF900895DF93CF930F92CDB7DEB78C
:104B100091E0998361E070E0AE014F5F5F4F0E94CA
:104B20000B2581E00F90CF91DF91089583E10E94E2
:104B30008325089582E10E94832508958AE00E94DA
:104B40008325089580E10E94832508958FE00E94C7
:104B50008325089589E00E94832508958EE00E94B0
:104B6000832508958DE00E94832508958BE00E949F
:104B7000832508958CE00E948325089583E00E9498
:104B8000832590E0089581E10E94832508958BE0BC
:104B90000E948325089587E00E94832590E0089570
:104BA00086E00E94832590E0089585E00E94832599
:104BB00090E0089584E00E94832590E0089582E0CB
:104BC0000E94832590E008950E9483250E94061983
:104BD000E0915B0CF0915C0C8191F0935C0CE093A4
:104BE0005B0C8D3321F083E08093460C0895E091B7
:104BF000520CF091530C89E78193F093530CE0939E
:104C0000520C81E00E94E11C08958DE10E94E42590
:104C100008958CE10E94E42508958BE10E94E4252B
:104C20000895CF93DF93C091520CD091530C86E33B
:104C300088838091520C9091530C01969093530C61
:104C40008093520C8AEE91E00E949C19892B19F0F6
:104C50000E94DF2595C08FEE91E00E949C19892B60
:104C600019F00E94DA258CC083EF91E00E949C1914
:104C7000892B19F00E94BE2583C088EF91E00E9425
:104C80009C19892B19F00E94D5257AC08CEF91E0F0
:104C90000E949C19892B19F00E94D02571C080E0D8
:104CA00092E00E949C19892B19F00E94CB2568C0C4
:104CB00084E092E00E949C19892B19F00E94AE2595
:104CC0005FC089E092E00E949C19892B19F00E9434
:104CD000B22556C08EE092E00E949C19892B19F0F3
:104CE0000E94B6254DC082E192E00E949C19892B5A
:104CF00019F00E94A62544C089E192E00E949C1907
:104D0000892B19F00E94A2253BC080E292E00E940C
:104D10009C19892B19F00E94AA2532C085E292E0E5
:104D20000E949C19892B19F00E94C32529C08AE290
:104D300092E00E949C19892B19F00E949A2520C0AC
:104D400080E392E00E949C19892B19F00E9496251D
:104D500017C086E392E00E949C19892B19F00E94EB
:104D60009E250EC08AE392E00E949C19892B19F0BF
:104D70000E94BA2505C0D093530CC093520C80E01A
:104D8000DF91CF9108951F93CF93DF93DB01EC0167
:104D90008A816AE00E94DE3E805DFD0181938A8106
:104DA0000E94DE3E905D11969C93DF0111961AE3FE
:104DB0001183AD014F5F5F4F89810E94DE3E805DB0
:104DC00011968C93FA01319689810E94DE3E905DA6
:104DD000DA0111969C93DF0111961183FD01319642
:104DE00088810E94DE3E805D11968C9388810E94AE
:104DF000DE3E905D91831282DF91CF911F910895E5
:104E000008950895E091520CF091530C80818E37F3
:104E100019F08F3761F406C03196F093530CE0938C
:104E2000520C08953296F093530CE093520C08956F
:104E300088E59FE09093530C8093520C0E940227C8
:104E40001DC00E940227E091520CF091530C8191F9
:104E5000F093530CE093520C90E001979C01220FC9
:104E6000331F280F391F220F331F220F331F2C51DE
:104E7000354FF90185919491FC010995E091520C0F
:104E8000F091530C80818D3721F08091460C88235E
:104E9000C1F208958AE08093540F8091510C8823C9
:104EA00071F01092510C89E38093460C8091760545
:104EB000909177059093570F8093560F81E0089556
:104EC0000F931F93DF93CF9300D0CDB7DEB70E942F
:104ED0007F2D8091BF059091C0059A8389838E01B3
:104EE0000F5F1F4F03C0C8010E945520E981FA815E
:104EF00080818823C1F70F900F90CF91DF911F9190
:104F00000F9108950E9460271092510C1092550F36
:104F10008AE08093540F1092430C10925F06109217
:104F20005E060895DF93CF93CDB7DEB764970FB6D3
:104F3000F894DEBF0FBECDBF2091560C3091570CB8
:104F400080917205909173052817390791F080EFD1
:104F500097E10E94C20DCE0101960E94010E898147
:104F6000893711F0893549F40E94942D8EED97E12F
:104F700002C086EC97E10E94C20D64960FB6F894C9
:104F8000DEBF0FBECDBFCF91DF91089507C0319630
:104F9000F0937804E09377040E94E10DE0917704A8
:104FA000F091780480818D3791F708950F931F93C6
:104FB000CF93DF93A0917704B0917804FD01219104
:104FC000F0937804E09377042633F1F1273330F43B
:104FD0002A3021F12C3009F04DC026C02E37D1F0F7
:104FE0002F3721F0243409F045C01BC011968C9155
:104FF0003196F0937804E0937704C0E0D0E0082F76
:1050000010E004C080E20E94E10D2196C017D10794
:10501000CCF340C080E20E94E10D3CC08DE498E1F9
:1050200005C08BE498E102C086E498E10E94C20DBD
:1050300080917704909178040196909378048093FE
:1050400077040E94C62726C011962C913196F093C2
:105050007804E093770430E021503040C901880F94
:10506000991F820F931F880F991F880F991F8A50CD
:10507000964F0EC030E021503040C901880F991F73
:10508000820F931F880F991F880F991F8A51954F80
:105090000E94C20DDF91CF911F910F9108951F9330
:1050A00090E00196E0917704F0917804E80FF91F01
:1050B000F0937804E09377041191F0937804E093EF
:1050C00077040CC0E0917704F09178048191F0931B
:1050D0007804E09377040E94E10D1150112391F7B9
:1050E0001F91089580E00E944F28089584E00E9457
:1050F0004F28089584E00E944F2808950F931F932E
:10510000CF93DF93E0917704F091780481819281CD
:105110003396F0937804E0937704C091BF05D09163
:10512000C005C80FD91F8E01025F1F4F89818823D8
:1051300011F00E94E10D2196C017D107B9F7DF9158
:10514000CF911F910F9108950E947E280895E091BC
:10515000520CF091530C82819F01280F311D309326
:105160007705209376058191919190935E0C8093C1
:105170005D0CF093530CE093520C80916B058823E7
:1051800089F08BE50E94E10D60915D0C70915E0CE1
:1051900080E090E00E94B0218DE50E94E10D80E268
:1051A0000E94E10D0895E0917704F0917804618107
:1051B00072813396F0937804E0937704882777FD23
:1051C0008095982F0E94B02108955CC00E94A72866
:1051D0008091520C9091530C01969093530C8093B4
:1051E000520C3AC00E940227E091520CF091530CED
:1051F0008191F093530CE093520C8F3041F40E9454
:105200003E378091460C882309F041C082E190E04E
:1052100001979C01220F331F280F391F220F331FC4
:10522000220F331F2C51354FF90185919491FC01C8
:1052300009958091460C882351F58091540F88235D
:1052400019F081508093540F8091540F882321F4DA
:105250000E944A278823D9F4E091520CF091530C14
:1052600080818D3709F0BECF9F012F5F3F4F809126
:105270007205909173052817390749F03093530C44
:105280002093520C8091460C882309F49FCF0895F7
:105290008091430C882359F48091560F9091570FB9
:1052A0009093530C8093520C0E94E528089585E258
:1052B0008093460C0E942A2208950E94770D0E9436
:1052C000822781E080934E062091560C3091570C36
:1052D00080917205909173052817390729F487E2A8
:1052E00098E10E94C20D08953093530C2093520C04
:1052F00030937705209376050E94E5288091460C2F
:10530000882311F00E942A220E94770D08950F939E
:105310001F93DF93CF93CDB7DEB72F970FB6F894D7
:10532000DEBF0FBECDBFE0917704F091780481819C
:1053300092813396F0937804E09377048E010F5FA7
:105340001F4FB8010E94CE0FC8010E94D50D2F96A5
:105350000FB6F894DEBF0FBECDBFCF91DF911F9186
:105360000F910895E0917704F0917804E081E93895
:1053700070F4E13821F0E238D9F1E43819F40E94F0
:105380007E280895E33869F50E9487290895E93A4F
:1053900060F5E13A19F40E947A280895E23A19F486
:1053A0000E9472280895E83A19F40E94D3280895BB
:1053B000E43A19F40E9476280895E43991F40E94A1
:1053C0007E2807C0E7FF03C00E94B22902C00E94E6
:1053D000D627E0917704F0917804E081ED3791F7DA
:1053E000089588E08093460C089588E08093460CE9
:1053F00008956F927F928F929F92AF92BF92CF92B9
:10540000DF92EF92FF920F931F93DF93CF93CDB76D
:10541000DEB7CF58D0400FB6F894DEBF0FBECDBF79
:105420000E94A818E0915B0CF0915C0C1081812F18
:1054300090E00E943D3F892B09F43EC180E492E058
:105440000E949C19892B09F43EC00E94770D86E4C6
:1054500092E00E94D50DEE24FF248E010F5F1F4FB6
:10546000C70165E070E00E94EA3E892B11F40E94BA
:10547000770DC701B8010E94CE0F8981882301F101
:10548000F80101900020E9F73197E01BF10B3E97FE
:1054900038F01F860EC0C80167E572E00E946F3FBA
:1054A000F80101900020E9F73197E01BF10B3E97DE
:1054B00090F3C8010E94D50D0894E11CF11CD0CFD7
:1054C0000E94770DF6C089E592E00E949C19892B15
:1054D00009F471C00E94770D1091BF050091C005BD
:1054E0008EE592E00E94D50D812F902F6C01760100
:1054F0000894E11CF11CAA24BB2490E1892E912C74
:1055000054C0C50183709070892B11F40E94770DEF
:10551000F60180818438D1F4C7010E94D50DF701CE
:1055200001900020E9F73197EE19FF0984010E1B65
:105530001F0B06C087E592E00E94D50D0150104078
:1055400001151105B9F783E792E024C0843909F009
:10555000B0C0C7010E94D50D88E792E00E94D50D2A
:105560008AE792E00E94D50DF70101900020E9F74B
:105570003197EE19FF0984010E1B1F0B06C087E54A
:1055800092E00E94D50D0150104001151105B9F7A8
:105590008CE792E00E94D50D0894A11CB11C83E118
:1055A00090E0C80ED91EE80EF91EF601808188230E
:1055B00009F0A7CF7EC08FE792E00E949C19892B4B
:1055C00009F473C0A0907704B0907804EE24FF240F
:1055D000870180E1882E912C8C0E9D1EB2E16B2EEE
:1055E000712C6C0E7D1E85E798E10E94C20DC801EA
:1055F000B7010E94B02182E798E10E94C20D8E2D72
:105600000E94E80EAB01BC01411551056105710511
:10561000A9F1C40120E830E00E94020FF401C0802B
:10562000D1807092780460927704FFEFCF16FFEF7D
:10563000DF0619F485E698E123C080E20E94E10DBF
:10564000B60180E090E00E94B021809177049091B3
:1056500078040196909378048093770407C0E7FF5D
:1056600003C00E94B22902C00E94D627E0917704AD
:10567000F0917804E081ED3791F704C081E598E17D
:105680000E94C20D0E94770D0894E11CF11C011DBF
:10569000111D83E0E816F1040105110509F0A3CFFF
:1056A000B0927804A092770404C085E892E00E944A
:1056B000D50D0E94770DACC0812F90E0C097E0918E
:1056C000560CF091570C20917205309173050A9792
:1056D000A0F5E217F30709F49BC00E94B618909357
:1056E0006506809364060E94A818E0915B0CF09117
:1056F0005C0C80818D32C1F43196F0935C0CE093A8
:105700005B0C0E94A818E0915B0CF0915C0C80810E
:1057100090E0C0970A9718F40E94B61809C08091CB
:10572000500F9091510F04C08091640690916506CE
:105730009093500680934F0612C0E217F30709F4C6
:1057400067C08091500F9091510F909350068093B5
:105750004F06808191819093650680936406209125
:1057600064063091650680914F069091500682172D
:10577000930708F44DC0C9010E94B02D909378049E
:10578000809377040E94770DE0917704F09178047C
:105790008091720590917305E817F907C8F501919A
:1057A0001191F0937804E093770480914F069091E3
:1057B00050068017910760F180E20E94E10DB80168
:1057C00080E090E00E94B02180917704909178046D
:1057D0000196909378048093770407C0E7FF03C095
:1057E0000E94B22902C00E94D627E0917704F0916E
:1057F0007804E081ED3791F70E94770D809177046E
:105800009091780401969093780480937704BCCFAC
:10581000C157DF4F0FB6F894DEBF0FBECDBFCF919B
:10582000DF911F910F91FF90EF90DF90CF90BF908D
:10583000AF909F908F907F906F900895DF92EF923E
:10584000FF920F931F937C018B01DC0113968C91C7
:1058500013976AE00E94DE3E805DF8018193139603
:105860008C910E94DE3E905DD80111969C9320E2BF
:10587000D22ED182CF0102966BEC72E00E947A3F69
:10588000F801D682D70115968C91159764E60E948F
:10589000DE3E892F6AE00E94DE3E805D878315969A
:1058A0008C9164E60E94DE3E892F6AE00E94DE3E13
:1058B000905D908711861F910F91FF90EF90DF9080
:1058C00008958FEC92E00E949C19892B19F00E9498
:1058D000F9294AC084ED92E00E949C19892B19F0A5
:1058E0000E945D2941C088ED92E00E949C19892B9D
:1058F00019F00E94922738C08CED92E00E949C190A
:10590000892B19F00E9448292FC081EE92E00E9455
:105910009C19892B19F00E94602726C087EE92E01F
:105920000E949C19892B19F00E94BB2C1DC08CEE83
:1059300092E00E949C19892B19F00E94A61214C0B3
:1059400081EF92E00E949C19892B19F00E94251585
:105950000BC086EF92E00E949C19892B19F420E07D
:1059600030E004C00E940C2D21E030E0C901089510
:105970000895089508950E94770D8DEC98E10E9496
:10598000C20D6091440C7091450C209172053091CC
:105990007305621B730B882777FD8095982F0E94F3
:1059A000B02181EC98E10E94C20D0E94770D8FEA30
:1059B00098E10E94C20D60914B0C70914C0C2091AB
:1059C0004E0F30914F0F621B730B882777FD809528
:1059D000982F0E94B02183EA98E10E94C20D0E9494
:1059E000770D84E898E10E94C20D60914A0F709192
:1059F0004B0F2091B7053091B805621B730B8827B8
:105A000077FD8095982F0E94B02188E798E10E9449
:105A1000C20D0E94770D08951F930E94A818E0916F
:105A20005B0CF0915C0C80818D3081F50E94ED1251
:105A3000182F8D3528F48A3558F48535C9F405C0FA
:105A40008F3FB1F481E699E152C08AE499E14FC0F9
:105A500084E399E10E94C20D1A3511F480E305C078
:105A60001B3511F481E301C082E30E94E10D0AC0FD
:105A70008BE199E10E94C20D612F70E080E090E01F
:105A80000E94B0218EE20E94E10D33C08DEF92E0C2
:105A90000E949C19892B19F08FEF90E023C081E0C0
:105AA00093E00E949C19892B19F085E590E01AC0BB
:105AB00084E093E00E949C19892B19F08AE590E01C
:105AC00011C088E093E00E949C19892B19F08BE5A6
:105AD00090E008C08CE093E00E949C19892B29F08B
:105AE0008CE590E00E940D1704C08EED98E10E94B5
:105AF000C20D1F910895089508950895089584EEA4
:105B00009CE06BE774E04CE30E942F1880EE9CE071
:105B100069E975E04EE10E94351810926C0510920B
:105B2000510610925A0C08950E94E70C1092510FE2
:105B30001092500F1092BE050895FB01E80FF91F57
:105B4000DB0102C081918D93809172059091730564
:105B5000E817F907B8F3B0937305A0937205089599
:105B60009C01E091560CF091570C80819181821735
:105B7000930714F0CF0108958281E80FF11DF5CF4E
:105B8000E091560CF091570C4091720550917305BD
:105B900020E030E00BC0208131812115310519F45E
:105BA00020E030E006C08281E80FF11DE417F50720
:105BB00091F7C90108959C018091500F9091510F68
:105BC00082179307A0F1E091560CF091570CDF017A
:105BD0004D915D914217530724F04217530739F551
:105BE00007C08281E82FF0E03297EA0FFB1FEFCF6A
:105BF0008C91DF01A80FB11D02C08D91819380911E
:105C0000720590917305A817B907B8F3F09373055F
:105C1000E09372058091500F9091510F48175907EA
:105C200031F40E94C02D9093510F8093500F08952E
:105C3000A0917205B0917305FD01E80FF91F8091E5
:105C4000440C9091450C8E179F0720F489E08093B7
:105C5000460C0895F0937305E0937205615070400F
:105C600004C08C91808331971197A617B707C9F7A5
:105C70000895DC0180915A0F282F30E088E59FE0DD
:105C80009093530C8093520C0CC0E091520CF09105
:105C9000530C81918D93F093530CE093520C21504F
:105CA00030402115310589F70895CF93DF93EC013A
:105CB00080915A0F90E0BE010E94182E8091460CF0
:105CC000882319F4CE010E94392EDF91CF910895D7
:105CD000409172055091730580915A0F9A01280FD7
:105CE000311D8091440C9091450C8217930780F0F0
:105CF000CA010E94392E20915A0F8091720590910D
:105D00007305820F911D909373058093720508951A
:105D100089E08093460C0895CF93DF93EC018A814C
:105D2000282F30E080915A0F281B310921153105A9
:105D300001F137FF0CC088279927821B930BBE0106
:105D40000E94182E8091460C8823B1F412C0DE0107
:105D5000A20FB31FFE0102C08D9181938091720545
:105D600090917305A817B907B8F3F0937305E09302
:105D70007205CE010E94392EDF91CF910895CF9305
:105D8000DF9381E08093430C88E59FE09093530C70
:105D90008093520CC091580FD091590F8091500FA1
:105DA0009091510F8C179D0738F40E94682ED09364
:105DB000510FC093500F18C0E091560CF091570C42
:105DC000808191818C179D0724F0C817D90749F469
:105DD00004C08281E80FF11DF3CFCF010E948C2E09
:105DE00003C0CF010E94552EDF91CF91089590E01E
:105DF0000197FC01EE0FFF1FE80FF91FEE0FFF1FC9
:105E0000EE0FFF1FEC51F54F85919491009711F023
:105E1000FC0109950895EF92FF920F931F93CF9382
:105E2000DF932091E50C81E090E0821B9109880FBF
:105E3000991F880F991FC091E60CD091E70CC81BE1
:105E4000D90B288139814A815B81CA01AA27BB27E6
:105E5000F9010BB68BBF819190810BBE7C0100E0F4
:105E600010E02E5F3F4F4F4F5F4FCA01AA27BB275D
:105E7000F9010BB68BBF219130810BBEC901A0E0A7
:105E8000B0E0DC01992788278E0D9F1DA01FB11F50
:105E900088839983AA83BB83DF91CF911F910F9150
:105EA000FF90EF900895CF93DF932091E50C81E070
:105EB00090E0821B9109880F991F880F991FC0914C
:105EC000E60CD091E70CC81BD90B88819981AA8177
:105ED000BB819D0144275527FC010BB62BBF808158
:105EE0000BBE90E0A0E0B0E088839983AA83BB83D7
:105EF000DF91CF910895CF93DF932091E50C81E05E
:105F000090E0821B9109880F991F880F991FC091FB
:105F1000E60CD091E70CC81BD90B88819981AA8126
:105F2000BB819D0144275527FC010BB62BBF8191F6
:105F300090810BBEA0E0B0E088839983AA83BB83E5
:105F4000DF91CF9108952091E50C81E090E0821BD4
:105F50009109880F991F880F991FE091E60CF09125
:105F6000E70CE81BF90B80819181A281B3818095B8
:105F70009095A095B09580839183A283B383089573
:105F80002091E50C81E090E0821B9109880F991F18
:105F9000880F991FE091E60CF091E70CE81BF90BD4
:105FA00080819181909581959F4FAA2797FDA0951B
:105FB000BA2F80839183A283B383089589E280936B
:105FC000460C08956F927F928F929F92AF92BF92EC
:105FD000CF92DF92EF92FF920F931F93CF93DF93B5
:105FE00084EE9CE068E30E946818AC01CB01DA0102
:105FF0005C016D012091E50C81E090E0821B91092C
:10600000880F991F880F991FC091E60CD091E70C5B
:10601000C81BD90B288139814A815B81D7FE04C016
:10602000EE24FF24870126C039014A0171E0E72EE2
:10603000F12C012D112D19C0C50181709070892B93
:1060400041F0C801B7019301A4010E94BF3E7B014A
:106050008C01B301C4019301A4010E94BF3E3B0126
:106060004C01D594C794B794A794A114B104C1046A
:10607000D10411F7E882F9820A831B83DF91CF9163
:106080001F910F91FF90EF90DF90CF90BF90AF9056
:106090009F908F907F906F90089584EE9CE068E3CE
:1060A0000E9468184091E50C21E030E0241B310982
:1060B000220F331F220F331FE091E60CF091E70C03
:1060C000E21BF30B20813181428153812617370770
:1060D0004807590749F081E090E0A0E0B0E08083F4
:1060E0009183A283B3830895108211821282138256
:1060F000089584EE9CE068E30E9468184091E50CE6
:1061000021E030E0241B3109220F331F220F331FFF
:10611000E091E60CF091E70CE21BF30B208131815A
:1061200042815381261737074807590749F481E010
:1061300090E0A0E0B0E080839183A283B3830895D0
:106140001082118212821382089584EE9CE068E32B
:106150000E9468184091E50C21E030E0241B3109D1
:10616000220F331F220F331FE091E60CF091E70C52
:10617000E21BF30B208131814281538126173707BF
:10618000480759074CF081E090E0A0E0B0E0808340
:106190009183A283B38308951082118212821382A5
:1061A000089584EE9CE068E30E9468184091E50C35
:1061B00021E030E0241B3109220F331F220F331F4F
:1061C000E091E60CF091E70CE21BF30B20813181AA
:1061D0004281538162177307840795074CF081E071
:1061E00090E0A0E0B0E080839183A283B383089520
:1061F0001082118212821382089584EE9CE068E37B
:106200000E9468184091E50C21E030E0241B310920
:10621000220F331F220F331FE091E60CF091E70CA1
:10622000E21BF30B20813181428153816217730796
:10623000840795074CF481E090E0A0E0B0E0808313
:106240009183A283B38308951082118212821382F4
:10625000089584EE9CE068E30E9468184091E50C84
:1062600021E030E0241B3109220F331F220F331F9E
:10627000E091E60CF091E70CE21BF30B20813181F9
:106280004281538126173707480759074CF481E0AC
:1062900090E0A0E0B0E080839183A283B38308956F
:1062A000108211821282138208950F931F9384EE3D
:1062B0009CE068E30E9468189B01AC016091E50CCA
:1062C00081E090E0861B9109880F991F880F991F24
:1062D0000091E60C1091E70C081B190BF801608186
:1062E0007181828193810E94BF3EF8016083718336
:1062F000828393831F910F9108950F931F9384EED0
:106300009CE068E30E9468189B01AC016091E50C79
:1063100081E090E0861B9109880F991F880F991FD3
:106320000091E60C1091E70C081B190BF801608135
:106330007181828193810E94203FF8016083718383
:10634000828393831F910F91089584EE9CE068E30C
:106350000E9468184091E50C21E030E0241B3109CF
:10636000220F331F220F331FE091E60CF091E70C50
:10637000E21BF30B2081318142815381261B370BB5
:10638000480B590B2083318342835383089584EE55
:106390009CE068E30E9468184091E50C21E030E041
:1063A000241B3109220F331F220F331FE091E60C0B
:1063B000F091E70CE21BF30B208131814281538184
:1063C000260F371F481F591F208331834283538371
:1063D000089584EE9CE068E30E9468184091E50C03
:1063E00021E030E0241B3109220F331F220F331F1D
:1063F000E091E60CF091E70CE21BF30B2081318178
:106400004281538126233723482359232083318314
:1064100042835383089584EE9CE068E30E946818E9
:106420004091E50C21E030E0241B3109220F331F9D
:10643000220F331FE091E60CF091E70CE21BF30B07
:106440002081318142815381262B372B482B592BB8
:106450002083318342835383089584EE9CE068E374
:106460000E9468184091E50C21E030E0241B3109BE
:10647000220F331F220F331FE091E60CF091E70C3F
:10648000E21BF30B2081318142815381262737277C
:10649000482759272083318342835383089584EE0C
:1064A0009CE068E30E946818CB010895CF92DF92C8
:1064B000EF92FF920F931F9384EE9CE068E30E949B
:1064C00068186B017C01C114D104E104F104F9F0F6
:1064D0002091E50C81E090E0821B9109880F991FC3
:1064E000880F991F0091E60C1091E70C081B190BFF
:1064F000F8016081718182819381A70196010E94D8
:10650000203FF801208331834283538305C08AE111
:106510008093460C0E942A221F910F91FF90EF90CA
:10652000DF90CF9008950F931F93682F80EE9CE02B
:1065300047E10E944E183DC08091460C8823F1F53A
:10654000E091E20CF091E30CE90FF11D42915291C0
:106550004031A1F1242F30E0207F3070852F90E072
:10656000807F9070821793074CF1413169F450316C
:1065700059F480EE9CE068E30E943B1880EE9CE0BA
:1065800068E30E943B181AC080EE9CE068E30E941A
:106590003B18082F80EE9CE068E30E943B18182F00
:1065A00080EE9CE0602F47E10E944E18812F0E94F0
:1065B000F72E9091E10C923008F0BECF1F910F9111
:1065C0000895893328F4873360F4813141F409C098
:1065D0008A3339F08A3318F08A57863010F080E019
:1065E000089581E10E94933281E00895CF93DF9373
:1065F000843861F0853820F4833809F081C070C098
:10660000843979F1843A09F07BC014C0E091520CCE
:10661000F091530C818192813396F093530CE09367
:10662000520C0F960E944A0DFC01408151816281FB
:1066300073816CC0E091520CF091530C41815281F6
:10664000638174813596F093530CE093520C359727
:1066500085813696E80FF11DF093530CE093520CB0
:1066600055C0E091520CF091530C81819281339688
:10667000F093530CE093520C0F960E944A0DFC01CC
:10668000C081D1818091520C9091530C01969093CE
:10669000530C8093520C0E948E338091520C909137
:1066A000530C01969093530C8093520C84EE9CE013
:1066B00068E30E946818FB0188819981E817F9074F
:1066C00020F089E18093460C26C0EE0FFF1FEE0FED
:1066D000FF1FEC0FFD1F428153816481758116C03D
:1066E000E091520CF091530C818192813396F0939A
:1066F000530CE093520C0E948A0EAB01BC0106C001
:1067000088E08093460C0E942A2205C084EE9CE01B
:1067100027E10E948818DF91CF9108951F9380E1AF
:106720000E9493320E940227E091520CF091530C88
:106730008081803141F43196F093530CE093520CF8
:106740000E948E3318C087FF07C00E94F6328091E6
:10675000460C882339F319C00E943336182F8091D4
:10676000460C882391F4812F0E94E132882369F43A
:10677000812F0E9493328091520C9091530C01967C
:106780009093530C8093520CCDCF1F910895EF92AC
:10679000FF920F931F93CF93DF930E948E3320912C
:1067A000E50C81E090E0821B9109880F991F880F0A
:1067B000991FC091E60CD091E70CC81BD90BE8805B
:1067C000F9800A811B81E114F1040105110569F4C6
:1067D0008EE491E6ACEBB0E080931003909311034C
:1067E000A0931203B093130328C06091100370911B
:1067F000110380911203909113032DE036E649E1D5
:1068000050E00E94BF3E615A7C408149934C6093A6
:106810001003709311038093120390931303A80144
:1068200097010E94FE3E9B01AC012F5F3F4F4F4FEF
:106830005F4F288339834A835B83DF91CF911F9118
:106840000F91FF90EF900895AF92BF92CF92DF9299
:10685000EF92FF920F931F930E948E332091E50CCD
:1068600081E090E0821B9109880F991F880F991F82
:10687000E091E60CF091E70CE81BF90BA080B180E9
:10688000C280D380E12CF12C012DA0E41A2F07C087
:1068900072E016950795F794E7947A95D1F7AE14C0
:1068A000BF04C006D106A0F320E030E040E050E095
:1068B00024C0D801C701820F931FA41FB51FA816BB
:1068C000B906CA06DB0670F0A81AB90ACA0ADB0ABA
:1068D000D801C701880F991FAA1FBB1F280F391F96
:1068E0004A1F5B1F569547953795279582E0169569
:1068F0000795F794E7948A95D1F7E114F10401051F
:106900001105B9F62A153B054C055D0520F42F5FEE
:106910003F4F4F4F5F4F20833183428353831F91FB
:106920000F91FF90EF90DF90CF90BF90AF900895C0
:106930001F93DF93CF9300D000D0CDB7DEB7182FD1
:106940000E948E332091E50C81E090E0821B91093A
:10695000880F991F880F991FE091E60CF091E70CC2
:10696000E81BF90B6081718182819381123039F0CB
:10697000143071F0113099F40E9420140BC00E9461
:10698000151369837A838B839C830E94770D0EC0D5
:106990000E94391369837A838B839C8307C083E0C9
:1069A0008093460C19821A821B821C8229813A81AB
:1069B0004B815C816091E50C81E090E0861B910940
:1069C000880F991F880F991FE091E60CF091E70C52
:1069D000E81BF90B20833183428353830F900F9080
:1069E0000F900F90CF91DF911F91089584E00E9446
:1069F0009834089582E00E949834089581E00E94BE
:106A0000983408950E948E332091E50C81E090E047
:106A1000821B9109880F991F880F991FE091E60C3E
:106A2000F091E70CE81BF90BA081B1818D919D914C
:106A30000D90BC91A02D80839183A283B383089590
:106A40000E948E332091E50C81E090E0821B910939
:106A5000880F991F880F991FE091E60CF091E70CC1
:106A6000E81BF90BA081B1818D919C91A0E0B0E071
:106A700080839183A283B38308950E948E332091F3
:106A8000E50C81E090E0821B9109880F991F880F27
:106A9000991FE091E60CF091E70CE81BF90BA0813F
:106AA000B1818C9190E0A0E0B0E080839183A283DB
:106AB000B38308950E948E3308950E948E332091EF
:106AC000E50C81E090E0821B9109880F991F880FE7
:106AD000991FE091E60CF091E70CE81BF90B80811F
:106AE0009181A281B3810097A105B10529F410829B
:106AF0001182128213820895B7FF05C08FEF9FEFB6
:106B0000AFEFBFEF04C081E090E0A0E0B0E0808391
:106B10009183A283B38308950E948E332091E50C64
:106B200081E090E0821B9109880F991F880F991FBF
:106B3000E091E60CF091E70CE81BF90B2081318124
:106B400037FF03C0309521953F4FC901AA2797FD14
:106B5000A095BA2F80839183A283B3830895CF93A6
:106B6000DF93843861F0853820F4833809F06DC0F4
:106B70005CC08439D1F0843A09F067C014C0E09158
:106B8000520CF091530C818192813396F093530C07
:106B9000E093520C0F960E944A0DAC01662757FDF8
:106BA0006095762F58C08AE351C0E091520CF09165
:106BB000530C818192813396F093530CE093520CE5
:106BC0000F960E944A0DFC01C081D1818091520C28
:106BD0009091530C01969093530C8093520C0E9409
:106BE0008E338091520C9091530C01969093530CDC
:106BF0008093520C84EE9CE068E30E9468188881C0
:106C000099816817790720F089E18093460C28C0A4
:106C10002296660F771F660F771FC60FD71FAE012C
:106C2000662757FD6095762F16C0E091520CF091C3
:106C3000530C818192813396F093530CE093520C64
:106C40000E94120DAB01BC0106C088E08093460C87
:106C50000E942A2205C084EE9CE027E10E94881849
:106C6000DF91CF910895863309F071C0E091520C05
:106C7000F091530C3196F093530CE093520C3197F2
:106C800081813396F093530CE093520C33978A3002
:106C9000F1F18B3098F4853059F1863040F483302F
:106CA00021F18430F8F4823009F041C039C08730D6
:106CB000B9F1873000F18930D1F520C08F3009F16A
:106CC000803138F48D3061F18E3050F58B3079F5AC
:106CD00027C0813149F18131B8F08231D9F0833157
:106CE00031F51BC00E948C3522C00E9424341FC085
:106CF0000E94C7331CC00E945D3519C00E943D35FB
:106D000016C00E94203513C00E94023510C00E9498
:106D1000FE340DC00E94FA340AC00E94F63407C047
:106D200089E28093460C03C083810E94AF35809135
:106D3000520C9091530C01969093530C8093520CEB
:106D40000E940227E091520CF091530C808108952B
:106D5000E091520CF091530C8081E80FF11DF093FB
:106D6000530CE093520C0895E091520CF091530CA7
:106D70008081E80FF11DF093530CE093520C0895BD
:106D8000A091520CB091530CFD012191F093530C42
:106D9000E093520C243951F411962D913C911297A5
:106DA0001396B093530CA093520C18C0223819F4C8
:106DB00020E030E015C011968D919C911297FD0155
:106DC0003396233831F49C01F093530CE093520C2A
:106DD00007C0F093530CE093520C9C01215F3F4F8E
:106DE000C9010895E0915106EE2321F48DE18093CD
:106DF000460C0895E150E0935106F0E0EE0FFF1FBE
:106E0000E852F04F808191819093530C8093520C03
:106E1000089508950895CF93DF93E0915A0CEE23DF
:106E200031F48FE18093460C0E942A2224C0C09145
:106E3000520CD091530CF0E0EE0FFF1FEA58FA4FBE
:106E4000808191819093530C8093520C0E948E33D9
:106E500084EE9CE068E30E94681861157105810565
:106E6000910549F4D093530CC093520C80915A0C65
:106E7000815080935A0CDF91CF910895CF93DF9387
:106E80000E940227C091520CD091530C8091BE05F4
:106E9000882351F08091720590917305019790932A
:106EA000530C8093520C06C02396D093530CC0937E
:106EB000520C23970E94022720915106203121F481
:106EC0008CE18093460C13C0E22FF0E0EE0FFF1F21
:106ED000E852F04F8091520C9091530C9183808333
:106EE0002F5F20935106D093530CC093520CDF9127
:106EF000CF9108950E94770D81E08093430C10920A
:106F00005E0C10925D0C8091720590917305019753
:106F10009093530C8093520C0895CF93DF9320915C
:106F20005A0C203131F48EE18093460C0E942A22C3
:106F300041C0E22FF0E0EE0FFF1FE858FA4F8091BA
:106F4000520C9091530C918380832F5F20935A0CA5
:106F5000C1E0D0E0E0917605F0917705F093530C15
:106F6000E093520C309731F1809172059091730546
:106F7000E817F90719F40E947A371CC082819F0133
:106F8000280F311D30937705209376053396F093C3
:106F9000530CE093520C0E940227E091520CF091A6
:106FA000530CE081E93111F42196D4CFEA3191F606
:106FB000219781F6DF91CF91089588E799E10E94AA
:106FC000C20D60915D0C70915E0C80E090E00E94BB
:106FD000B0211092430C80917605909177059093A3
:106FE000570F8093560F10925E0C10925D0C80919B
:106FF00072059091730501979093530C8093520CF6
:1070000008950E940227E091520CF091530C2181C7
:1070100032813396F093530CE093520C5091BE059D
:10702000552341F0809172059091730590937705F7
:1070300080937605E0917605F09177056091720571
:1070400070917305E617F70721F4E091560CF09163
:10705000570C808191812817390720F4E091560C54
:10706000F091570C8081918182179307B1F4F093CE
:10707000530CE093520C552341F01092BE0581E071
:1070800080934E060E94E52808953396F093530CA2
:10709000E093520C0E940227089542812817390775
:1070A00028F0E40FF11DE617F707E1F68BE1809376
:1070B000460C0895AF92BF92CF92DF92EF92FF926B
:1070C0000F931F93CF93DF93E091520CF091530CE9
:1070D0001081103731F0133721F0143711F000E030
:1070E0000DC03196F093530CE093520C0E9402278E
:1070F000E091520CF091530C012F10810E94C03688
:107100007C01143919F0C0E0D0E034C08091520CF9
:107110009091530C01969093530C8093520C0E94C3
:107120008E338091520C9091530C01969093530C96
:107130008093520C8091460C882309F082C0C701CD
:107140000E944A0DFC01C081D18184EE9CE068E37D
:107150000E946818888199816817790720F089E171
:107160008093460C6EC02296660F771F660F771FBE
:10717000C60FD71F0E9402278091520C9091530C8A
:1071800001969093530C8093520C0E948E33809101
:10719000460C882309F055C084EE9CE068E30E9409
:1071A00068185B016C01133831F4C701B601A50101
:1071B0000E94490E46C0143929F4688379838A8372
:1071C0009B833FC0C7010E944A0DFC010023D9F0F8
:1071D0002081318142815381003749F4CA01AA27B5
:1071E000BB27F9010BB68BBFA0820BBE2AC00437A8
:1071F00079F4CA01AA27BB27F9010BB68BBFA1926C
:10720000B0820BBE1EC09C01442737FD4095542F11
:10721000CA01AA27BB27F9010BB68BBFA192B08286
:107220000BBE2E5F3F4F4F4F5F4F7A010027112754
:10723000C601AA27BB27F9010BB6EBBE8193908349
:107240000BBEDF91CF911F910F91FF90EF90DF90D8
:10725000CF90BF90AF9008958FEF80936B05089506
:1072600010926B05089508958091520C9091530CE3
:1072700003969093530C8093520C0E948E3380910E
:10728000520C9091530C01969093530C8093520C96
:1072900008951F93182F82958F708A3008F0895FA8
:1072A000805D0E94E10D812F8F708A3008F0895F28
:1072B000805D0E94E10D1F910895EF92FF920F9360
:1072C0001F930E94343984EE9CE068E30E946818A2
:1072D0007B018C01892F9927AA27BB270E94493956
:1072E000C801AA27BB270E944939BB27A12F902F8D
:1072F0008F2D0E9449398E2D0E9449391F910F917F
:10730000FF90EF900895EF92FF920F931F930E94CA
:10731000343984EE9CE068E30E9468187B018C019C
:10732000BB27A92F982F872F0E9449398E2D0E94A5
:1073300049391F910F91FF90EF9008950E943439C1
:1073400084EE9CE068E30E946818862F0E94493909
:1073500008950E94343984EE9CE068E30E94681826
:10736000862F0E94E10D08950E94343984EE9CE03E
:1073700068E30E94681889E00E94E10D0895EF9289
:10738000FF920F931F930E940227E091520CF091FD
:10739000530CE08110E07BC0EB37B1F1EC3720F407
:1073A000E63309F05FC03BC0EC3759F1E23A09F02F
:1073B00059C0E091520CF091530C6181E62EFF24EC
:1073C00000E010E08EEF9FEFAFEFBFEFE80EF91E89
:1073D0000A1F1B1F3396F093530CE093520CCF01FE
:1073E000B7010E94093DB7016F5F7F4F8091520C3A
:1073F0009091530C860F971F9093530C8093520CCF
:1074000023C089E00E94E10D8091520C9091530CB1
:1074100001969093530C8093520C11E031C0E0918F
:10742000520CF091530C81818B3099F08C3028F400
:10743000823061F08730B1F405C08D3069F08E3054
:1074400089F40DC00E94B43910E01AC00E94A93915
:1074500028C00E945D3925C00E949E3922C00E942A
:1074600083391FC00E948E338091460C8823E9F433
:1074700084EE9CE068E30E9468180E94B02111C06D
:107480000E940227E091520CF091530CE081ED37FD
:1074900019F0EA3709F080CF112339F40E94770DF3
:1074A00004C080E20E94E10DCFCF1F910F91FF90A9
:1074B000EF900895EF92FF920F931F93CF93DF9376
:1074C000E090B705F090B8050E940227E091520CB9
:1074D000F091530C808184FD02C081E22FC0818134
:1074E00092810F960E944A0DEC018091520C90916E
:1074F000530C04969093530C8093520C0E948E333D
:107500008091520C9091530C01969093530C809360
:10751000520C88819981AA81BB810097A105B10590
:1075200009F047C00091B7051091B80584EE9CE0C2
:1075300068E30E94681877FF04C087E28093460CD6
:1075400047C04091B7055091B805198308831B8245
:107550001A826F5F7F4FF801718360834E5F5F4FC8
:10756000CB01880F991F880F991F840F951F4250D8
:1075700050409093B8058093B70520914A0F309101
:107580004B0F2817390720F0FA0180E090E00EC079
:1075900089E08093460CF092B805E092B70518C0D8
:1075A00012821382148215820196349686179707E9
:1075B000B8F30E940227E091520CF091530C8081A5
:1075C0008D3731F03196F093530CE093520C78CF15
:1075D000DF91CF911F910F91FF90EF900895089543
:1075E00008950895089508950895089508950895B3
:1075F000089508958091BE05882329F083E3809340
:10760000460C0E942A220895CF93DF93C091520C1A
:10761000D091530C8091560C9091570C9093530C31
:107620008093520C90935F0680935E06E091520C1B
:10763000F091530C82819F01280F311D30935F061A
:1076400020935E063396F093530CE093520C0E9405
:107650000227E091520CF091530C80818C3051F450
:107660003296F0935F06E0935E06D093530CC0937E
:10767000520C1AC020915E0630915F06809172050F
:10768000909173052817390751F4D093530CC09388
:10769000520C86E28093460C0E942A2205C0309349
:1076A000530C2093520CC2CFDF91CF910895CF930A
:1076B000DF93C091520CD091530C80915E06909153
:1076C0005F069093530C8093520C8091520C9091D2
:1076D000530C03969093530C8093520C0E940227F4
:1076E000E091520CF091530C80818C3051F4339620
:1076F000F0935F06E0935E06D093530CC093520C58
:107700001BC0E0915E06F0915F068091720590913A
:107710007305E817F90741F4D093530CC093520C4A
:1077200086E28093460C08C08281E80FF11DF09339
:107730005F06E0935E06C9CFDF91CF910895CF92A7
:10774000DF92EF92FF920F931F930E9402270E94F5
:10775000C0368C010E94E90DC82EC8010E944A0D56
:10776000FC01DD24EE24FF24C082D182E282F38278
:107770001F910F91FF90EF90DF90CF900895CF93DE
:10778000DF930E9402270E94C0369C0190916C05F5
:107790008EE0989FE0011124CD54DA4F88819981C1
:1077A0002817390731F084E28093460C0E942A2280
:1077B00045C0C9010E944A0DFC01208131814281EE
:1077C00053818A819B81AC81BD81280F391F4A1F5B
:1077D0005B1F20833183428353838A819B81AC81E9
:1077E000BD81B7FF0AC08E819F81A885B985281702
:1077F00039074A075B07B4F40DC00097A105B1052E
:1078000089F08E819F81A885B98582179307A40787
:10781000B50744F480916C05815080936C050E94FB
:1078200002270CC08A859B859093530C8093520C41
:107830008C859D8590935E0C80935D0CDF91CF913C
:107840000895DF92EF92FF920F931F93D82E8091AD
:10785000520C9091530C01969093530C8093520CC0
:107860000E9402270E948E330E9402278091520CB0
:107870009091530C01969093530C8093520C0E945C
:1078800002278091520C9091530C01969093530CC7
:107890008093520C0E948E3384EE9CE068E30E9439
:1078A00068187B018C0184EE9CE068E30E946818F4
:1078B00022E0D216A1F034E0D316F9F041E0D4165C
:1078C00011F580E090E02FEF30E040E050E0E22260
:1078D000F322042315234E2D0E94BF1714C080E00D
:1078E00090E02FEF3FEF40E050E0E222F32204234C
:1078F0001523A7010E947E1706C080E090E0A80132
:1079000097010E9497171F910F91FF90EF90DF90C2
:10791000089584E00E94213C089582E00E94213C69
:10792000089581E00E94213C08950E948E330E94B8
:1079300002278091520C9091530C01969093530C16
:107940008093520C0E94022784EE9CE068E30E9420
:1079500068189B01AC018091460C8823C1F5E09129
:10796000520CF091530C232B31F08081883A79F539
:107970000E94013808958081883A79F43396F09313
:10798000530CE093520C0E940227E091520CF091AC
:10799000530C80818933D9F40AC080917605909187
:1079A000770501979093530C8093520C089531966C
:1079B000F093530CE093520C0E940227E091520C7A
:1079C000F091530C8081883A11F40E940138089597
:1079D0001F93E0915B0CF0915C0C80818D3211F073
:1079E00010E006C03196F0935C0CE0935B0C11E064
:1079F0000E94DB1E9B01AC01112339F0509540958C
:107A0000309521953F4F4F4F5F4FB901CA011F91EC
:107A100008950F931F93CF93DF938C01EB0106C062
:107A2000F80181918F010E94860D21972097C1F75F
:107A3000DF91CF911F910F910895EF92FF920F93D5
:107A40001F93E0915B0CF0915C0C8081843241F4D7
:107A50003196F0935C0CE0935B0C0E947F1F02C098
:107A60000E94E83C7B018C010E94A818E0915B0C0D
:107A7000F0915C0C80818D3071F08C3231F4319654
:107A8000F0935C0CE0935B0C06C085E18093460CA0
:107A90000E942A2209C00E94C0360E944A0DFC01A1
:107AA000E082F182028313831F910F91FF90EF9088
:107AB00008950E94A818E0915B0CF0915C0C808105
:107AC0008D30C9F00E941D3D8091460C882399F4A9
:107AD0000E940227E091520CF091530C80818D3767
:107AE00069F08A3759F03196F093530CE093520CB9
:107AF0000E940227DECF21E030E002C020E030E02B
:107B0000C901089580915E0690915F06892B21F44A
:107B10000E94043B0E94573B80915E0690915F0655
:107B200090935C0C80935B0C0E9402270E94593D4D
:107B300020915B0C30915C0C019769F42E5F3F4FF4
:107B400030935F0620935E060E94573B8091460C5F
:107B5000882311F304C030935F0620935E060895D6
:107B6000EF92FF920F931F930E940227E091520C15
:107B7000F091530C8081823A01F5018110E00250AE
:107B8000104083E0E82EF12CEE0EFF1EC701B80175
:107B90000E94093D0F5F1F4FE00EF11EF092530C43
:107BA000E092520C0E9402278091520C9091530C4B
:107BB00001969093530C8093520C0E9402278FE3FE
:107BC0000E94E10D80E20E94E10D0E94081B0E94CC
:107BD000770D0E944A27882321F40E94593D892B62
:107BE00071F71092F80F1F910F91FF90EF90089589
:107BF0000F931F9380916C058A3031F483E2809358
:107C0000460C0E942A22B8C00E9402270091520C02
:107C10001091530C0E94C03640916C05242F30E027
:107C2000220F331FF90173E0EE0FFF1F7A95E1F782
:107C3000E21BF30BEF53FA4F91838083842F90E084
:107C4000880F991FFC0153E0EE0FFF1F5A95E1F7D3
:107C5000E81BF90BEF53FA4F80915D0C90915E0C8D
:107C6000958784871093530C0093520C0E945A38C6
:107C70000E9402278091520C9091530C0196909390
:107C8000530C8093520C0E9402270E948E33109155
:107C90006C0584EE9CE068E30E946818212F30E0B8
:107CA000220F331FF90103E0EE0FFF1F0A95E1F7E2
:107CB000E21BF30BEF53FA4F66837783808791873C
:107CC00080916C0590E0FC0113E0EE0FFF1F1A9508
:107CD000E1F7E81BF90BEE0FFF1FED53FA4F81E0C0
:107CE00090E0A0E0B0E080839183A283B3830E9400
:107CF0000227E091520CF091530C80818A3319F5E0
:107D00003196F093530CE093520C0E9402270E948C
:107D10008E3300916C0510E084EE9CE068E30E94D5
:107D20006818F801A3E0EE0FFF1FAA95E1F7E01B2A
:107D3000F10BEE0FFF1FED53FA4F608371838283C7
:107D400093830E94022720916C05822F90E0880F78
:107D5000991FFC0133E0EE0FFF1F3A95E1F7E81B96
:107D6000F90BEF53FA4F8091520C9091530C93877B
:107D700082872F5F20936C051F910F910895629F5A
:107D8000D001739FF001829FE00DF11D649FE00D13
:107D9000F11D929FF00D839FF00D749FF00D659F74
:107DA000F00D9927729FB00DE11DF91F639FB00D73
:107DB000E11DF91FBD01CF0111240895991B79E040
:107DC00004C0991F961708F0961B881F7A95C9F76B
:107DD00080950895AA1BBB1B51E107C0AA1FBB1FBA
:107DE000A617B70710F0A61BB70B881F991F5A9547
:107DF000A9F780959095BC01CD010895A1E21A2EB6
:107E0000AA1BBB1BFD010DC0AA1FBB1FEE1FFF1F3E
:107E1000A217B307E407F50720F0A21BB30BE40B8E
:107E2000F50B661F771F881F991F1A9469F76095D5
:107E30007095809590959B01AC01BD01CF0108958F
:107E400097FB092E05260ED057FD04D0D7DF0AD0A8
:107E5000001C38F450954095309521953F4F4F4F79
:107E60005F4F0895F6F790958095709561957F4FD7
:107E70008F4F9F4F089585FD59C08062911156C064
:107E800081568A51E0F70895911150C080538A506D
:107E900028F0865C806281568650B8F7089591116B
:107EA000089581548A5108F4805E855A089591118D
:107EB000089581568A5108F4805285580895FB012F
:107EC000DC0105900D920020E1F70895FC0105907A
:107ED0000020E9F7809590958E0F9F1F0895FB0174
:107EE000DC010D900020E9F7119701900D92002020
:107EF000E1F70895FB01DC0101900D920020E1F70C
:107F00000895F999FECF92BD81BDF89A992780B561
:107F10000895262FF999FECF92BD81BD20BD0FB6E1
:107F2000F894FA9AF99A0FBE01960895992788272E
:067F30000895F894FFCF54
:107F3600010102014201430183018401646174610C
:107F4600006C6574007265616400726573746F72AB
:107F56006500676F73756200676F746F006F6E0000
:107F660072657475726E00696600696E707574006C
:107F76007072696E7400666F72006E657874007355
:107F8600746F7000656E64776800656E6400726574
:107F96006D0064696D0074726F6E0074726F666650
:107FA600007768696C6500656570313600656570D7
:107FB60033320065657000696E62797465003F0052
:107FC6002700656C7365003C3D003E3D003C3E006D
:107FD6003C003E003D00414E44004F5200454F528A
:107FE600002B002D002A002F006D6F64005E0040FC
:107FF6003136004033320040006E6F7400746F00FB
:1080060053544550007468656E00656C736500478F
:108016004F544F00474F5355420043485224006186
:108026006273007371727400524E440053474E00DF
:1080360054414200686578340068657832006865A6
:1080460078007065656B3136007065656B3332009C
:108056007065656B00616464720065657031360039
:108066006565703332006565700074696D6524005E
:10807600706F727473004C697374206F6620706F32
:10808600727473202D2D00200076617273004C6986
:108096007374206F66207661726961626C65732005
:1080A6002D2D0020202020002800290020200066F9
:1080B600696C657300556E6B6E6F776E204C495315
:1080C6005420746F7069632E202054727920276CB7
:1080D60069737420706F72747327206F7220276C17
:1080E600697374207661727327206F7220276C691A
:1080F60073742066696C6573272E006D6F6E006C55
:108106006973740072756E006E657700636F6E74C6
:1081160000636C6561720066726565006C6F616410
:108126000073617665006175746F7374006F6666BF
:1081360000656500666C3000666C3100666C320066
:048146004E61BC00CA
:020000021000EC
:10FC0000AF92BF92CF92DF92EF92FF920F931F932A
:10FC1000CF93DF937B018C016A01AFB6F894F99919
:10FC2000FECF07B600FCFDCF83E0F70100935B0039
:10FC300080935700E89507B600FCFDCF40E050E008
:10FC400060E070E0BB24B394F6018081D181C0E014
:10FC50009E01280F311D82E090E0C80ED91EDB0105
:10FC6000CA018E0D9F1DA01FB11F0901FC01A093A9
:10FC70005B00B0925700E89511244E5F5F4F6F4FC5
:10FC80007F4F403091E0590790E0690790E0790795
:10FC9000D9F685E0F70100935B0080935700E89563
:10FCA00007B600FCFDCF81E180935700E895AFBE19
:10FCB000DF91CF911F910F91FF90EF90DF90CF9048
:06FCC000BF90AF90089513
:00000001FF
